:020000020000FC
:100000000C94A3030C942A000C942A000C942A004C
:100010000C942A000C942A000C942A000C942A00B8
:100020000C942A000C942A000C942A000C942A00A8
:100030000C942A000C942A000C942A000C942A0098
:100040000C942A000C942A000C942A000C942A0088
:100050000C942A0018956A95F1F7089560E570E010
:10006000609360007093610060E070E060936200F4
:10007000709363000895FF91EF91EE0FFF1F65915C
:1000800075918091600090916100791738F011F0BE
:10009000BC0104C0681710F009F0BC016093620055
:1000A00070936300C4E6D0E08591899361507040FD
:1000B000D9F7F695E795EF93FF93089560E0F62E54
:1000C00060E4E62E60E8D62E60ECC62EF5BA6FEF3F
:1000D00064BB0895F5BA6DE90E942B00F5BA67E09C
:1000E0000E942B00E5BA67E00E942B00F5BA089544
:1000F000D5BA6DE90E942B00D5BA67E00E942B00AB
:10010000C5BA67E00E942B00D5BA08958F938F730C
:100110008D938F9108958F93883008F48EE28F37F6
:1001200008F08EE280FB869587F98D938F91089574
:10013000CF93DF938F93C4E6D0E06091620070911B
:1001400063008C918F3B41F48D918C918F3F11F422
:10015000A4EBB0E08D918D9189910E948B0061504C
:10016000704079F78F91DF91CF9108958F93969A90
:100170008E98A4EBB0E079E183E00E9486008BE1E9
:100180000E9486008FE00E9486008FE30E94860016
:100190008CE30E94860068E28EE20E948B006A95E2
:1001A000D9F78FEB8D937A9539F78FEF8D938F91E8
:1001B0000895193168F4953058F4A4EBB0E06EE27C
:1001C000169FA00DB11DA90F90E0B91F0C948600D9
:1001D00008951931E8F70832D8F7A9EBB0E06EE2DC
:1001E000169FA00DB11DA00F70E0B71F0C948B00DF
:1001F000193170F7083260F7A9EBB0E06EE2169F94
:10020000A00DB11DA00F70E0B71F0C949800BD9019
:10021000AD909D908D907D90ED91FE2FFF73E078D5
:10022000E72B099466E00E942B00E5BA67E00E9484
:100230002B00F5BA08950E94070167E00E942B0089
:10024000000000009E97869B0C94070162E00E94CC
:100250002B00000000000C946A0070E027E0DE0133
:100260000E941B0165E00E942B00705F70772A9549
:10027000B1F70000DE0100000C941B01C4EBD0E0DC
:1002800039E13A950E942D0163E00E942B00AE9661
:100290003A95C1F7000000000C942D012BE00E945C
:1002A0006A006DE00E942B0000002A95C1F7000053
:1002B00000000C946A002CE00E9478006DE00E941F
:1002C0002B0000002A95C1F7000000000C94780074
:1002D00028E10E946A006DE00E942B0000002A9530
:1002E000C1F7000000000C946A000E943E016CE01F
:1002F0000E942B00000000000E944E016CE00E9452
:100300002B00000000000E945B016CE00E942B00AB
:100310000000000000000C9468010E9475010000BC
:100320000000000000000000000000000000F5CF09
:1003300080E090E00E94D9000E943B00280020202D
:1003400020202020202020202020202020202020AD
:10035000202020202020202020202020202020209D
:100360002020202020200E94F8001395089510E0FE
:1003700000E00E943B002800202020202021222392
:100380002425262728292A2B2C2D2E2F30313233B5
:100390003435363738393A3B3C3D3E3F202020202B
:1003A0000E94F80013950E943B0028002020202086
:1003B000404142434445464748494A4B4C4D4E4FC5
:1003C000505152535455565758595A5B5C5D5E5FB5
:1003D000202020200E94F80013950E943B00280056
:1003E00020202020606162636465666768696A6BCB
:1003F0006C6D6E6F707172737475767778797A7BC5
:100400007C7D7E20202020200E94F80013950E94F1
:1004100098010E943B0028002D2D2D2D2E5F2E2DA2
:10042000275F602D2D2D2D3C207B205B5D207D20C6
:100430003E2D2D2D2D2E5F2E2D275F602D2D2D2D48
:1004400080E390E00E94D90080E091E00E94D90012
:100450000E94F80013958CE390E00E94D90080E0A0
:1004600091E00E94D9000E94F80013958CE090E082
:100470000E94D90080E091E00E94D9000E94F8001B
:1004800013958FE090E00E94D90080E091E00E94F7
:10049000D9000E94F800139583E090E00E94D900F3
:1004A00080E091E00E94D9000E94F800139583E358
:1004B00090E00E94D90080E091E00E94D9000E9463
:1004C000F80013950E9498010E943B0028004156B5
:1004D000522041546D6567613332207543202B20D3
:1004E000536F6674564741203D203430306C696E3E
:1004F00065203730487A0E94F80013950E943B002F
:10050000280031382E3334324D487A2C2033636C36
:100510006B2F7069786C2C20347069786C2F63684D
:1005200061722C203430636861720E94F800139568
:100530000E943B00280066756C6C2041534349497A
:100540002C20347838706978656C20666F6E742C56
:100550002032206C696E65732F706978656C0E941B
:10056000F80013950E9498010E943B0028006E6FCE
:100570007208696E76096E6F720A756C696E0B6E21
:100580006F720C322F330C6E6F720D312F330D6E74
:100590006F720E70617380E090E00E94D90083E07A
:1005A00091E00E94D90082E092E00E94D90081E0AF
:1005B00093E00E94D9008BE294E00E94D9000E944F
:1005C000F800139580E090E00E94D9008CE091E063
:1005D0000E94D90088E092E00E94D90084E093E074
:1005E0000E94D9008EE294E00E94D9000E94F80097
:1005F000139580E090E00E94D9008FE091E00E9486
:10060000D9008AE092E00E94D90085E093E00E9440
:10061000D9008FE294E00E94D9000E94F80013955F
:1006200080E090E00E94D90080E391E00E94D90030
:1006300080E292E00E94D90080E193E00E94D9001C
:100640008AE394E00E94D9000E94F800139580E0AC
:1006500090E00E94D90083E391E00E94D90082E2F9
:1006600092E00E94D90081E193E00E94D9008BE3DF
:1006700094E00E94D9000E94F800139580E090E079
:100680000E94D9008CE391E00E94D90088E292E0B8
:100690000E94D90084E193E00E94D9008EE394E0A7
:1006A0000E94D9000E94F800139580E090E00E941B
:1006B000D9008FE391E00E94D9008AE292E00E9483
:1006C000D90085E193E00E94D9008FE394E00E9475
:1006D000D9000E94F80013950E9498010E943B00E7
:1006E000280064657369676E20616E6420636F64BF
:1006F00065206F70656E20736F757263652061761B
:1007000061696C61626C652061740E94F8001395E8
:100710000E943B002800687474703A2F2F6E656940
:100720006C2E6672616E6B6C696E2E63682F5072F0
:100730006F6A656374732F536F66745647410E94E6
:10074000F800139508956FE578E06DBF7EBF78944B
:100750000E942E000E945E000E94B6000E94B70117
:02076000DCCDEE
:10080000B5BA6A2CAB2CB62CED91FE2FFF73E078B5
:10081000E0600994000000000000000000000000FB
:10082000B5BA6A2CAB2CB62CED91FE2FFF73E07895
:10083000E0610994000000000000000000000000DA
:10084000B5BA6A2CAB2CB62CED91FE2FFF73E07875
:10085000E0620994000000000000000000000000B9
:10086000B5BA6A2CAB2CB62CED91FE2FFF73E07855
:10087000E063099400000000000000000000000098
:10088000B5BA6A2CAB2CB62CED91FE2FFF73E07835
:10089000E064099400000000000000000000000077
:1008A000B5BA6A2CAB2CB62CED91FE2FFF73E07815
:1008B000E065099400000000000000000000000056
:1008C000B5BA6A2CAB2CB62CED91FE2FFF73E078F5
:1008D000E066099400000000000000000000000035
:1008E000B5BA6A2CAB2CB62CED91FE2FFF73E078D5
:1008F000E067099400000000000000000000000014
:10090000A5BA6A2CAB2CB62CED91FE2FFF73E078C4
:10091000E0600994000000000000000000000000FA
:10092000A5BA6A2CAB2CB62CED91FE2FFF73E078A4
:10093000E0610994000000000000000000000000D9
:10094000A5BA6A2CAB2CB62CED91FE2FFF73E07884
:10095000E0620994000000000000000000000000B8
:10096000A5BA6A2CAB2CB62CED91FE2FFF73E07864
:10097000E063099400000000000000000000000097
:10098000A5BA6A2CAB2CB62CED91FE2FFF73E07844
:10099000E064099400000000000000000000000076
:1009A000A5BA6A2CAB2CB62CED91FE2FFF73E07824
:1009B000E065099400000000000000000000000055
:1009C000A5BA6A2CAB2CB62CED91FE2FFF73E07804
:1009D000E066099400000000000000000000000034
:1009E000A5BA6A2CAB2CB62CED91FE2FFF73E078E4
:1009F000E067099400000000000000000000000013
:100A0000B5BA000000000000ED91FE2FFF73E07802
:100A1000E0600994000000000000000000000000F9
:100A2000B5BA000000000000ED91FE2FFF73E078E2
:100A3000E0610994000000000000000000000000D8
:100A4000B5BA000000000000ED91FE2FFF73E078C2
:100A5000E0620994000000000000000000000000B7
:100A6000B5BA000000000000ED91FE2FFF73E078A2
:100A7000E063099400000000000000000000000096
:100A8000B5BA000000000000ED91FE2FFF73E07882
:100A9000E064099400000000000000000000000075
:100AA000B5BA000000000000ED91FE2FFF73E07862
:100AB000E065099400000000000000000000000054
:100AC000B5BA000000000000ED91FE2FFF73E07842
:100AD000E066099400000000000000000000000033
:100AE000B5BA6A2CAB2CB62CED91FE2FFF73E078D3
:100AF000E067099400000000000000000000000012
:100B0000B5BA000000000000ED91FE2FFF73E07801
:100B1000E0600994000000000000000000000000F8
:100B2000B5BA000000000000ED91FE2FFF73E078E1
:100B3000E0610994000000000000000000000000D7
:100B4000B5BA000000000000ED91FE2FFF73E078C1
:100B5000E0620994000000000000000000000000B6
:100B6000B5BA000000000000ED91FE2FFF73E078A1
:100B7000E063099400000000000000000000000095
:100B8000B5BA000000000000ED91FE2FFF73E07881
:100B9000E064099400000000000000000000000074
:100BA000B5BA000000000000ED91FE2FFF73E07861
:100BB000E065099400000000000000000000000053
:100BC000B5BA000000000000ED91FE2FFF73E07841
:100BD000E066099400000000000000000000000032
:100BE000A5BA6A2CAB2CB62CED91FE2FFF73E078E2
:100BF000E067099400000000000000000000000011
:100C0000B5BA6A2CA92C962CED91FE2FFF73E078D3
:100C1000E0600994000000000000000000000000F7
:100C2000B5BA6A2CA92C962CED91FE2FFF73E078B3
:100C3000E0610994000000000000000000000000D6
:100C4000B5BA6A2CA92C962CED91FE2FFF73E07893
:100C5000E0620994000000000000000000000000B5
:100C6000B5BA6A2CA92C962CED91FE2FFF73E07873
:100C7000E063099400000000000000000000000094
:100C8000B5BA6A2CA92C962CED91FE2FFF73E07853
:100C9000E064099400000000000000000000000073
:100CA000B5BA6A2CA92C962CED91FE2FFF73E07833
:100CB000E065099400000000000000000000000052
:100CC000B5BA6A2CA92C962CED91FE2FFF73E07813
:100CD000E066099400000000000000000000000031
:100CE000B5BA6A2CA92C962CED91FE2FFF73E078F3
:100CF000E067099400000000000000000000000010
:100D0000B5BA6A2CA82C862CED91FE2FFF73E078E3
:100D1000E0600994000000000000000000000000F6
:100D2000B5BA6A2CA82C862CED91FE2FFF73E078C3
:100D3000E0610994000000000000000000000000D5
:100D4000B5BA6A2CA82C862CED91FE2FFF73E078A3
:100D5000E0620994000000000000000000000000B4
:100D6000B5BA6A2CA82C862CED91FE2FFF73E07883
:100D7000E063099400000000000000000000000093
:100D8000B5BA6A2CA82C862CED91FE2FFF73E07863
:100D9000E064099400000000000000000000000072
:100DA000B5BA6A2CA82C862CED91FE2FFF73E07843
:100DB000E065099400000000000000000000000051
:100DC000B5BA6A2CA82C862CED91FE2FFF73E07823
:100DD000E066099400000000000000000000000030
:100DE000B5BA6A2CA82C862CED91FE2FFF73E07803
:100DF000E06709940000000000000000000000000F
:100E0000B5BA6A2CA72C762CED91FE2FFF73E078F3
:100E1000E0600994000000000000000000000000F5
:100E2000B5BA6A2CA72C762CED91FE2FFF73E078D3
:100E3000E0610994000000000000000000000000D4
:100E4000B5BA6A2CA72C762CED91FE2FFF73E078B3
:100E5000E0620994000000000000000000000000B3
:100E6000B5BA6A2CA72C762CED91FE2FFF73E07893
:100E7000E063099400000000000000000000000092
:100E8000B5BA6A2CA72C762CED91FE2FFF73E07873
:100E9000E064099400000000000000000000000071
:100EA000B5BA6A2CA72C762CED91FE2FFF73E07853
:100EB000E065099400000000000000000000000050
:100EC000B5BA6A2CA72C762CED91FE2FFF73E07833
:100ED000E06609940000000000000000000000002F
:100EE000B5BA6A2CA72C762CED91FE2FFF73E07813
:100EF000E06709940000000000000000000000000E
:10100000B5BAED91B5BAFE2FFF73B5BAE078E060DE
:10101000B5BA0994000000000000000000000000C4
:10102000B5BAED91B5BAFE2FFF73B5BAE078E061BD
:10103000B5BA0994000000000000000000000000A4
:10104000B5BAED91B5BAFE2FFF73B5BAE078E0629C
:10105000B5BA099400000000000000000000000084
:10106000B5BAED91B5BAFE2FFF73B5BAE078E0637B
:10107000B5BA099400000000000000000000000064
:10108000B5BAED91B5BAFE2FFF73B5BAE078E0645A
:10109000B5BA099400000000000000000000000044
:1010A000B5BAED91B5BAFE2FFF73B5BAE078E06539
:1010B000B5BA099400000000000000000000000024
:1010C000B5BAED91B5BAFE2FFF73B5BAE078E06618
:1010D000B5BA099400000000000000000000000004
:1010E000B5BAED91B5BAFE2FFF73B5BAE078E067F7
:1010F000B5BA0994000000000000000000000000E4
:10110000B5BAED91B5BAFE2FFF73B5BAE078E060DD
:10111000B5BA0994000000000000000000000000C3
:10112000B5BAED91B5BAFE2FFF73B5BAE078E061BC
:10113000B5BA0994000000000000000000000000A3
:10114000B5BAED91B5BAFE2FFF73B5BAE078E0629B
:10115000B5BA099400000000000000000000000083
:10116000B5BAED91B5BAFE2FFF73B5BAE078E0637A
:10117000B5BA099400000000000000000000000063
:10118000B5BAED91B5BAFE2FFF73B5BAE078E06459
:10119000B5BA099400000000000000000000000043
:1011A000B5BAED91B5BAFE2FFF73B5BAE078E06538
:1011B000B5BA099400000000000000000000000023
:1011C000B5BAED91B5BAFE2FFF73B5BAE078E06617
:1011D000B5BA099400000000000000000000000003
:1011E000B5BAED91B5BAFE2FFF73B5BAE078E067F6
:1011F000B5BA0994000000000000000000000000E3
:10120000B5BAED91B5BAFE2FFF73B5BAE078E060DC
:10121000B5BA0994000000000000000000000000C2
:10122000B5BAED91B5BAFE2FFF73B5BAE078E061BB
:10123000B5BA0994000000000000000000000000A2
:10124000B5BAED91B5BAFE2FFF73B5BAE078E0629A
:10125000B5BA099400000000000000000000000082
:10126000B5BAED91B5BAFE2FFF73B5BAE078E06379
:10127000B5BA099400000000000000000000000062
:10128000B5BAED91B5BAFE2FFF73B5BAE078E06458
:10129000B5BA099400000000000000000000000042
:1012A000B5BAED91B5BAFE2FFF73B5BAE078E06537
:1012B000B5BA099400000000000000000000000022
:1012C000B5BAED91B5BAFE2FFF73B5BAE078E06616
:1012D000B5BA099400000000000000000000000002
:1012E000B5BAED91B5BAFE2FFF73B5BAE078E067F5
:1012F000B5BA0994000000000000000000000000E2
:10130000B5BAED91B5BAFE2FFF73B5BAE078E060DB
:10131000B5BA0994000000000000000000000000C1
:10132000B5BAED91B5BAFE2FFF73B5BAE078E061BA
:10133000B5BA0994000000000000000000000000A1
:10134000B5BAED91B5BAFE2FFF73B5BAE078E06299
:10135000B5BA099400000000000000000000000081
:10136000B5BAED91B5BAFE2FFF73B5BAE078E06378
:10137000B5BA099400000000000000000000000061
:10138000B5BAED91B5BAFE2FFF73B5BAE078E06457
:10139000B5BA099400000000000000000000000041
:1013A000B5BAED91B5BAFE2FFF73B5BAE078E06536
:1013B000B5BA099400000000000000000000000021
:1013C000B5BAED91B5BAFE2FFF73B5BAE078E06615
:1013D000B5BA099400000000000000000000000001
:1013E000B5BAED91B5BAFE2FFF73B5BAE078E067F4
:1013F000B5BA0994000000000000000000000000E1
:10140000B5BAED91B5BAFE2FFF73B5BAE078E060DA
:10141000B5BA0994000000000000000000000000C0
:10142000B5BAED91B5BAFE2FFF73B5BAE078E061B9
:10143000B5BA0994000000000000000000000000A0
:10144000B5BAED91B5BAFE2FFF73B5BAE078E06298
:10145000B5BA099400000000000000000000000080
:10146000B5BAED91B5BAFE2FFF73B5BAE078E06377
:10147000B5BA099400000000000000000000000060
:10148000B5BAED91B5BAFE2FFF73B5BAE078E06456
:10149000B5BA099400000000000000000000000040
:1014A000B5BAED91B5BAFE2FFF73B5BAE078E06535
:1014B000B5BA099400000000000000000000000020
:1014C000B5BAED91B5BAFE2FFF73B5BAE078E06614
:1014D000B5BA099400000000000000000000000000
:1014E000B5BAED91B5BAFE2FFF73B5BAE078E067F3
:1014F000B5BA0994000000000000000000000000E0
:10150000B5BAED91B5BAFE2FFF73B5BAE078E060D9
:10151000B5BA0994000000000000000000000000BF
:10152000B5BAED91B5BAFE2FFF73B5BAE078E061B8
:10153000B5BA09940000000000000000000000009F
:10154000B5BAED91B5BAFE2FFF73B5BAE078E06297
:10155000B5BA09940000000000000000000000007F
:10156000B5BAED91B5BAFE2FFF73B5BAE078E06376
:10157000B5BA09940000000000000000000000005F
:10158000B5BAED91B5BAFE2FFF73B5BAE078E06455
:10159000B5BA09940000000000000000000000003F
:1015A000B5BAED91B5BAFE2FFF73B5BAE078E06534
:1015B000B5BA09940000000000000000000000001F
:1015C000B5BAED91B5BAFE2FFF73B5BAE078E06613
:1015D000B5BA0994000000000000000000000000FF
:1015E000B5BAED91B5BAFE2FFF73B5BAE078E067F2
:1015F000B5BA0994000000000000000000000000DF
:10160000B5BAED91B5BAFE2FFF73B5BAE078E060D8
:10161000B5BA0994000000000000000000000000BE
:10162000B5BAED91B5BAFE2FFF73B5BAE078E061B7
:10163000B5BA09940000000000000000000000009E
:10164000B5BAED91B5BAFE2FFF73B5BAE078E06296
:10165000B5BA09940000000000000000000000007E
:10166000B5BAED91B5BAFE2FFF73B5BAE078E06375
:10167000B5BA09940000000000000000000000005E
:10168000B5BAED91B5BAFE2FFF73B5BAE078E06454
:10169000B5BA09940000000000000000000000003E
:1016A000B5BAED91B5BAFE2FFF73B5BAE078E06533
:1016B000B5BA09940000000000000000000000001E
:1016C000B5BAED91B5BAFE2FFF73B5BAE078E06612
:1016D000B5BA0994000000000000000000000000FE
:1016E000B5BAED91B5BAFE2FFF73B5BAE078E067F1
:1016F000B5BA0994000000000000000000000000DE
:10170000B5BAED91B5BAFE2FFF73B5BAE078E060D7
:10171000B5BA0994000000000000000000000000BD
:10172000B5BAED91B5BAFE2FFF73B5BAE078E061B6
:10173000B5BA09940000000000000000000000009D
:10174000B5BAED91B5BAFE2FFF73B5BAE078E06295
:10175000B5BA09940000000000000000000000007D
:10176000B5BAED91B5BAFE2FFF73B5BAE078E06374
:10177000B5BA09940000000000000000000000005D
:10178000B5BAED91B5BAFE2FFF73B5BAE078E06453
:10179000B5BA09940000000000000000000000003D
:1017A000B5BAED91B5BAFE2FFF73B5BAE078E06532
:1017B000B5BA09940000000000000000000000001D
:1017C000B5BAED91B5BAFE2FFF73B5BAE078E06611
:1017D000B5BA0994000000000000000000000000FD
:1017E000B5BAED91B5BAFE2FFF73B5BAE078E067F0
:1017F000B5BA0994000000000000000000000000DD
:10180000B5BAED91B5BAFE2FFF73B5BAE078E060D6
:10181000B5BA0994000000000000000000000000BC
:10182000B5BAED91B5BAFE2FFF73B5BAE078E061B5
:10183000B5BA09940000000000000000000000009C
:10184000B5BAED91B5BAFE2FFF73B5BAE078E06294
:10185000B5BA09940000000000000000000000007C
:10186000B5BAED91B5BAFE2FFF73B5BAE078E06373
:10187000B5BA09940000000000000000000000005C
:10188000B5BAED91B5BAFE2FFF73B5BAE078E06452
:10189000B5BA09940000000000000000000000003C
:1018A000B5BAED91B5BAFE2FFF73B5BAE078E06531
:1018B000B5BA09940000000000000000000000001C
:1018C000B5BAED91B5BAFE2FFF73B5BAE078E06610
:1018D000B5BA0994000000000000000000000000FC
:1018E000B5BAED91B5BAFE2FFF73B5BAE078E067EF
:1018F000B5BA0994000000000000000000000000DC
:10190000B5BAED91B5BAFE2FFF73B5BAE078E060D5
:10191000B5BA0994000000000000000000000000BB
:10192000B5BAED91B5BAFE2FFF73B5BAE078E061B4
:10193000B5BA09940000000000000000000000009B
:10194000B5BAED91B5BAFE2FFF73B5BAE078E06293
:10195000B5BA09940000000000000000000000007B
:10196000B5BAED91B5BAFE2FFF73B5BAE078E06372
:10197000B5BA09940000000000000000000000005B
:10198000B5BAED91B5BAFE2FFF73B5BAE078E06451
:10199000B5BA09940000000000000000000000003B
:1019A000B5BAED91B5BAFE2FFF73B5BAE078E06530
:1019B000B5BA09940000000000000000000000001B
:1019C000B5BAED91B5BAFE2FFF73B5BAE078E0660F
:1019D000B5BA0994000000000000000000000000FB
:1019E000B5BAED91B5BAFE2FFF73B5BAE078E067EE
:1019F000B5BA0994000000000000000000000000DB
:101A0000B5BAED91B5BAFE2FFF73B5BAE078E060D4
:101A1000B5BA0994000000000000000000000000BA
:101A2000B5BAED91B5BAFE2FFF73B5BAE078E061B3
:101A3000B5BA09940000000000000000000000009A
:101A4000B5BAED91B5BAFE2FFF73B5BAE078E06292
:101A5000B5BA09940000000000000000000000007A
:101A6000B5BAED91B5BAFE2FFF73B5BAE078E06371
:101A7000B5BA09940000000000000000000000005A
:101A8000B5BAED91B5BAFE2FFF73B5BAE078E06450
:101A9000B5BA09940000000000000000000000003A
:101AA000B5BAED91B5BAFE2FFF73B5BAE078E0652F
:101AB000B5BA09940000000000000000000000001A
:101AC000B5BAED91B5BAFE2FFF73B5BAE078E0660E
:101AD000B5BA0994000000000000000000000000FA
:101AE000B5BAED91B5BAFE2FFF73B5BAE078E067ED
:101AF000B5BA0994000000000000000000000000DA
:101B0000B5BAED91B5BAFE2FFF73B5BAE078E060D3
:101B1000B5BA0994000000000000000000000000B9
:101B2000B5BAED91B5BAFE2FFF73B5BAE078E061B2
:101B3000B5BA099400000000000000000000000099
:101B4000B5BAED91B5BAFE2FFF73B5BAE078E06291
:101B5000B5BA099400000000000000000000000079
:101B6000B5BAED91B5BAFE2FFF73B5BAE078E06370
:101B7000B5BA099400000000000000000000000059
:101B8000B5BAED91B5BAFE2FFF73B5BAE078E0644F
:101B9000B5BA099400000000000000000000000039
:101BA000B5BAED91B5BAFE2FFF73B5BAE078E0652E
:101BB000B5BA099400000000000000000000000019
:101BC000B5BAED91B5BAFE2FFF73B5BAE078E0660D
:101BD000B5BA0994000000000000000000000000F9
:101BE000B5BAED91B5BAFE2FFF73B5BAE078E067EC
:101BF000B5BA0994000000000000000000000000D9
:101C0000B5BAED91B5BAFE2FFF73B5BAE078E060D2
:101C1000B5BA0994000000000000000000000000B8
:101C2000B5BAED91B5BAFE2FFF73B5BAE078E061B1
:101C3000B5BA099400000000000000000000000098
:101C4000B5BAED91B5BAFE2FFF73B5BAE078E06290
:101C5000B5BA099400000000000000000000000078
:101C6000B5BAED91B5BAFE2FFF73B5BAE078E0636F
:101C7000B5BA099400000000000000000000000058
:101C8000B5BAED91B5BAFE2FFF73B5BAE078E0644E
:101C9000B5BA099400000000000000000000000038
:101CA000B5BAED91B5BAFE2FFF73B5BAE078E0652D
:101CB000B5BA099400000000000000000000000018
:101CC000B5BAED91B5BAFE2FFF73B5BAE078E0660C
:101CD000B5BA0994000000000000000000000000F8
:101CE000B5BAED91B5BAFE2FFF73B5BAE078E067EB
:101CF000B5BA0994000000000000000000000000D8
:101D0000B5BAED91B5BAFE2FFF73B5BAE078E060D1
:101D1000B5BA0994000000000000000000000000B7
:101D2000B5BAED91B5BAFE2FFF73B5BAE078E061B0
:101D3000B5BA099400000000000000000000000097
:101D4000B5BAED91B5BAFE2FFF73B5BAE078E0628F
:101D5000B5BA099400000000000000000000000077
:101D6000B5BAED91B5BAFE2FFF73B5BAE078E0636E
:101D7000B5BA099400000000000000000000000057
:101D8000B5BAED91B5BAFE2FFF73B5BAE078E0644D
:101D9000B5BA099400000000000000000000000037
:101DA000B5BAED91B5BAFE2FFF73B5BAE078E0652C
:101DB000B5BA099400000000000000000000000017
:101DC000B5BAED91B5BAFE2FFF73B5BAE078E0660B
:101DD000B5BA0994000000000000000000000000F7
:101DE000B5BAED91B5BAFE2FFF73B5BAE078E067EA
:101DF000B5BA0994000000000000000000000000D7
:101E0000B5BAED91B5BAFE2FFF73B5BAE078E060D0
:101E1000B5BA0994000000000000000000000000B6
:101E2000B5BAED91B5BAFE2FFF73B5BAE078E061AF
:101E3000B5BA099400000000000000000000000096
:101E4000B5BAED91B5BAFE2FFF73B5BAE078E0628E
:101E5000B5BA099400000000000000000000000076
:101E6000B5BAED91B5BAFE2FFF73B5BAE078E0636D
:101E7000B5BA099400000000000000000000000056
:101E8000B5BAED91B5BAFE2FFF73B5BAE078E0644C
:101E9000B5BA099400000000000000000000000036
:101EA000B5BAED91B5BAFE2FFF73B5BAE078E0652B
:101EB000B5BA099400000000000000000000000016
:101EC000B5BAED91B5BAFE2FFF73B5BAE078E0660A
:101ED000B5BA0994000000000000000000000000F6
:101EE000B5BAED91B5BAFE2FFF73B5BAE078E067E9
:101EF000B5BA0994000000000000000000000000D6
:101F0000B5BAED91B5BAFE2FFF73B5BAE078E060CF
:101F1000B5BA0994000000000000000000000000B5
:101F2000B5BAED91B5BAFE2FFF73B5BAE078E061AE
:101F3000B5BA099400000000000000000000000095
:101F4000B5BAED91B5BAFE2FFF73B5BAE078E0628D
:101F5000B5BA099400000000000000000000000075
:101F6000B5BAED91B5BAFE2FFF73B5BAE078E0636C
:101F7000B5BA099400000000000000000000000055
:101F8000B5BAED91B5BAFE2FFF73B5BAE078E0644B
:101F9000B5BA099400000000000000000000000035
:101FA000B5BAED91B5BAFE2FFF73B5BAE078E0652A
:101FB000B5BA099400000000000000000000000015
:101FC000B5BAED91B5BAFE2FFF73B5BAE078E06609
:101FD000B5BA0994000000000000000000000000F5
:101FE000B5BAED91B5BAFE2FFF73B5BAE078E067E8
:101FF000B5BA0994000000000000000000000000D5
:10200000B5BAED91B5BAFE2FFF73B5BAE078E060CE
:10201000B5BA0994000000000000000000000000B4
:10202000B5BAED91B5BAFE2FFF73B5BAE078E061AD
:10203000B5BA099400000000000000000000000094
:10204000B5BAED91B5BAFE2FFF73B5BAE078E0628C
:10205000B5BA099400000000000000000000000074
:10206000B5BAED91B5BAFE2FFF73B5BAE078E0636B
:10207000B5BA099400000000000000000000000054
:10208000B5BAED91B5BAFE2FFF73B5BAE078E0644A
:10209000B5BA099400000000000000000000000034
:1020A000B5BAED91B5BAFE2FFF73B5BAE078E06529
:1020B000B5BA099400000000000000000000000014
:1020C000B5BAED91B5BAFE2FFF73B5BAE078E06608
:1020D000B5BA0994000000000000000000000000F4
:1020E000B5BAED91B5BAFE2FFF73B5BAE078E067E7
:1020F000B5BA0994000000000000000000000000D4
:10210000B5BAED91B5BAFE2FFF73B5BAE078E060CD
:10211000B5BA0994000000000000000000000000B3
:10212000B5BAED91A5BAFE2FFF73B5BAE078E061BC
:10213000B5BA099400000000000000000000000093
:10214000B5BAED91A5BAFE2FFF73B5BAE078E0629B
:10215000B5BA099400000000000000000000000073
:10216000B5BAED91A5BAFE2FFF73B5BAE078E0637A
:10217000B5BA099400000000000000000000000053
:10218000B5BAED91A5BAFE2FFF73B5BAE078E06459
:10219000B5BA099400000000000000000000000033
:1021A000B5BAED91B5BAFE2FFF73B5BAE078E06528
:1021B000B5BA099400000000000000000000000013
:1021C000B5BAED91A5BAFE2FFF73B5BAE078E06617
:1021D000B5BA0994000000000000000000000000F3
:1021E000B5BAED91B5BAFE2FFF73B5BAE078E067E6
:1021F000B5BA0994000000000000000000000000D3
:10220000B5BAED91B5BAFE2FFF73B5BAE078E060CC
:10221000B5BA0994000000000000000000000000B2
:10222000A5BAED91B5BAFE2FFF73A5BAE078E061CB
:10223000B5BA099400000000000000000000000092
:10224000A5BAED91B5BAFE2FFF73A5BAE078E062AA
:10225000B5BA099400000000000000000000000072
:10226000B5BAED91B5BAFE2FFF73B5BAE078E06369
:10227000B5BA099400000000000000000000000052
:10228000B5BAED91B5BAFE2FFF73B5BAE078E06448
:10229000B5BA099400000000000000000000000032
:1022A000B5BAED91B5BAFE2FFF73B5BAE078E06527
:1022B000B5BA099400000000000000000000000012
:1022C000B5BAED91B5BAFE2FFF73B5BAE078E06606
:1022D000B5BA0994000000000000000000000000F2
:1022E000B5BAED91B5BAFE2FFF73B5BAE078E067E5
:1022F000B5BA0994000000000000000000000000D2
:10230000B5BAED91B5BAFE2FFF73B5BAE078E060CB
:10231000B5BA0994000000000000000000000000B1
:10232000B5BAED91B5BAFE2FFF73B5BAE078E061AA
:10233000B5BA099400000000000000000000000091
:10234000A5BAED91B5BAFE2FFF73A5BAE078E062A9
:10235000B5BA099400000000000000000000000071
:10236000A5BAED91A5BAFE2FFF73A5BAE078E06398
:10237000B5BA099400000000000000000000000051
:10238000A5BAED91B5BAFE2FFF73A5BAE078E06467
:10239000B5BA099400000000000000000000000031
:1023A000A5BAED91A5BAFE2FFF73A5BAE078E06556
:1023B000B5BA099400000000000000000000000011
:1023C000A5BAED91B5BAFE2FFF73A5BAE078E06625
:1023D000B5BA0994000000000000000000000000F1
:1023E000B5BAED91B5BAFE2FFF73B5BAE078E067E4
:1023F000B5BA0994000000000000000000000000D1
:10240000B5BAED91B5BAFE2FFF73B5BAE078E060CA
:10241000B5BA0994000000000000000000000000B0
:10242000B5BAED91B5BAFE2FFF73B5BAE078E061A9
:10243000B5BA099400000000000000000000000090
:10244000B5BAED91A5BAFE2FFF73A5BAE078E062A8
:10245000B5BA099400000000000000000000000070
:10246000A5BAED91A5BAFE2FFF73B5BAE078E06387
:10247000B5BA099400000000000000000000000050
:10248000B5BAED91A5BAFE2FFF73B5BAE078E06456
:10249000B5BA099400000000000000000000000030
:1024A000B5BAED91A5BAFE2FFF73A5BAE078E06545
:1024B000B5BA099400000000000000000000000010
:1024C000A5BAED91A5BAFE2FFF73B5BAE078E06624
:1024D000B5BA0994000000000000000000000000F0
:1024E000B5BAED91B5BAFE2FFF73B5BAE078E067E3
:1024F000B5BA0994000000000000000000000000D0
:10250000B5BAED91B5BAFE2FFF73B5BAE078E060C9
:10251000B5BA0994000000000000000000000000AF
:10252000A5BAED91B5BAFE2FFF73A5BAE078E061C8
:10253000B5BA09940000000000000000000000008F
:10254000B5BAED91B5BAFE2FFF73A5BAE078E06297
:10255000B5BA09940000000000000000000000006F
:10256000B5BAED91A5BAFE2FFF73B5BAE078E06376
:10257000B5BA09940000000000000000000000004F
:10258000B5BAED91A5BAFE2FFF73B5BAE078E06455
:10259000B5BA09940000000000000000000000002F
:1025A000A5BAED91B5BAFE2FFF73B5BAE078E06534
:1025B000B5BA09940000000000000000000000000F
:1025C000A5BAED91B5BAFE2FFF73A5BAE078E06623
:1025D000B5BA0994000000000000000000000000EF
:1025E000B5BAED91B5BAFE2FFF73B5BAE078E067E2
:1025F000B5BA0994000000000000000000000000CF
:10260000B5BAED91B5BAFE2FFF73B5BAE078E060C8
:10261000B5BA0994000000000000000000000000AE
:10262000B5BAED91A5BAFE2FFF73B5BAE078E061B7
:10263000B5BA09940000000000000000000000008E
:10264000A5BAED91B5BAFE2FFF73A5BAE078E062A6
:10265000B5BA09940000000000000000000000006E
:10266000B5BAED91A5BAFE2FFF73B5BAE078E06375
:10267000B5BA09940000000000000000000000004E
:10268000A5BAED91B5BAFE2FFF73A5BAE078E06464
:10269000B5BA09940000000000000000000000002E
:1026A000A5BAED91B5BAFE2FFF73A5BAE078E06543
:1026B000B5BA09940000000000000000000000000E
:1026C000B5BAED91A5BAFE2FFF73A5BAE078E06622
:1026D000B5BA0994000000000000000000000000EE
:1026E000B5BAED91B5BAFE2FFF73B5BAE078E067E1
:1026F000B5BA0994000000000000000000000000CE
:10270000B5BAED91B5BAFE2FFF73B5BAE078E060C7
:10271000B5BA0994000000000000000000000000AD
:10272000B5BAED91A5BAFE2FFF73B5BAE078E061B6
:10273000B5BA09940000000000000000000000008D
:10274000A5BAED91B5BAFE2FFF73B5BAE078E06295
:10275000B5BA09940000000000000000000000006D
:10276000B5BAED91B5BAFE2FFF73B5BAE078E06364
:10277000B5BA09940000000000000000000000004D
:10278000B5BAED91B5BAFE2FFF73B5BAE078E06443
:10279000B5BA09940000000000000000000000002D
:1027A000B5BAED91B5BAFE2FFF73B5BAE078E06522
:1027B000B5BA09940000000000000000000000000D
:1027C000B5BAED91B5BAFE2FFF73B5BAE078E06601
:1027D000B5BA0994000000000000000000000000ED
:1027E000B5BAED91B5BAFE2FFF73B5BAE078E067E0
:1027F000B5BA0994000000000000000000000000CD
:10280000B5BAED91B5BAFE2FFF73B5BAE078E060C6
:10281000B5BA0994000000000000000000000000AC
:10282000B5BAED91A5BAFE2FFF73B5BAE078E061B5
:10283000B5BA09940000000000000000000000008C
:10284000A5BAED91B5BAFE2FFF73B5BAE078E06294
:10285000B5BA09940000000000000000000000006C
:10286000A5BAED91B5BAFE2FFF73B5BAE078E06373
:10287000B5BA09940000000000000000000000004C
:10288000A5BAED91B5BAFE2FFF73B5BAE078E06452
:10289000B5BA09940000000000000000000000002C
:1028A000A5BAED91B5BAFE2FFF73B5BAE078E06531
:1028B000B5BA09940000000000000000000000000C
:1028C000B5BAED91A5BAFE2FFF73B5BAE078E06610
:1028D000B5BA0994000000000000000000000000EC
:1028E000B5BAED91B5BAFE2FFF73B5BAE078E067DF
:1028F000B5BA0994000000000000000000000000CC
:10290000B5BAED91B5BAFE2FFF73B5BAE078E060C5
:10291000B5BA0994000000000000000000000000AB
:10292000B5BAED91A5BAFE2FFF73B5BAE078E061B4
:10293000B5BA09940000000000000000000000008B
:10294000B5BAED91B5BAFE2FFF73A5BAE078E06293
:10295000B5BA09940000000000000000000000006B
:10296000B5BAED91B5BAFE2FFF73A5BAE078E06372
:10297000B5BA09940000000000000000000000004B
:10298000B5BAED91B5BAFE2FFF73A5BAE078E06451
:10299000B5BA09940000000000000000000000002B
:1029A000B5BAED91B5BAFE2FFF73A5BAE078E06530
:1029B000B5BA09940000000000000000000000000B
:1029C000B5BAED91A5BAFE2FFF73B5BAE078E0660F
:1029D000B5BA0994000000000000000000000000EB
:1029E000B5BAED91B5BAFE2FFF73B5BAE078E067DE
:1029F000B5BA0994000000000000000000000000CB
:102A0000B5BAED91B5BAFE2FFF73B5BAE078E060C4
:102A1000B5BA0994000000000000000000000000AA
:102A2000B5BAED91B5BAFE2FFF73B5BAE078E061A3
:102A3000B5BA09940000000000000000000000008A
:102A4000B5BAED91A5BAFE2FFF73B5BAE078E06292
:102A5000B5BA09940000000000000000000000006A
:102A6000A5BAED91A5BAFE2FFF73A5BAE078E06391
:102A7000B5BA09940000000000000000000000004A
:102A8000B5BAED91A5BAFE2FFF73B5BAE078E06450
:102A9000B5BA09940000000000000000000000002A
:102AA000A5BAED91A5BAFE2FFF73A5BAE078E0654F
:102AB000B5BA09940000000000000000000000000A
:102AC000B5BAED91A5BAFE2FFF73B5BAE078E0660E
:102AD000B5BA0994000000000000000000000000EA
:102AE000B5BAED91B5BAFE2FFF73B5BAE078E067DD
:102AF000B5BA0994000000000000000000000000CA
:102B0000B5BAED91B5BAFE2FFF73B5BAE078E060C3
:102B1000B5BA0994000000000000000000000000A9
:102B2000B5BAED91B5BAFE2FFF73B5BAE078E061A2
:102B3000B5BA099400000000000000000000000089
:102B4000B5BAED91A5BAFE2FFF73B5BAE078E06291
:102B5000B5BA099400000000000000000000000069
:102B6000B5BAED91A5BAFE2FFF73B5BAE078E06370
:102B7000B5BA099400000000000000000000000049
:102B8000A5BAED91A5BAFE2FFF73A5BAE078E0646F
:102B9000B5BA099400000000000000000000000029
:102BA000B5BAED91A5BAFE2FFF73B5BAE078E0652E
:102BB000B5BA099400000000000000000000000009
:102BC000B5BAED91A5BAFE2FFF73B5BAE078E0660D
:102BD000B5BA0994000000000000000000000000E9
:102BE000B5BAED91B5BAFE2FFF73B5BAE078E067DC
:102BF000B5BA0994000000000000000000000000C9
:102C0000B5BAED91B5BAFE2FFF73B5BAE078E060C2
:102C1000B5BA0994000000000000000000000000A8
:102C2000B5BAED91B5BAFE2FFF73B5BAE078E061A1
:102C3000B5BA099400000000000000000000000088
:102C4000B5BAED91B5BAFE2FFF73B5BAE078E06280
:102C5000B5BA099400000000000000000000000068
:102C6000B5BAED91B5BAFE2FFF73B5BAE078E0635F
:102C7000B5BA099400000000000000000000000048
:102C8000B5BAED91B5BAFE2FFF73B5BAE078E0643E
:102C9000B5BA099400000000000000000000000028
:102CA000B5BAED91A5BAFE2FFF73B5BAE078E0652D
:102CB000B5BA099400000000000000000000000008
:102CC000B5BAED91A5BAFE2FFF73B5BAE078E0660C
:102CD000B5BA0994000000000000000000000000E8
:102CE000A5BAED91B5BAFE2FFF73B5BAE078E067EB
:102CF000B5BA0994000000000000000000000000C8
:102D0000B5BAED91B5BAFE2FFF73B5BAE078E060C1
:102D1000B5BA0994000000000000000000000000A7
:102D2000B5BAED91B5BAFE2FFF73B5BAE078E061A0
:102D3000B5BA099400000000000000000000000087
:102D4000B5BAED91B5BAFE2FFF73B5BAE078E0627F
:102D5000B5BA099400000000000000000000000067
:102D6000B5BAED91B5BAFE2FFF73B5BAE078E0635E
:102D7000B5BA099400000000000000000000000047
:102D8000A5BAED91A5BAFE2FFF73A5BAE078E0646D
:102D9000B5BA099400000000000000000000000027
:102DA000B5BAED91B5BAFE2FFF73B5BAE078E0651C
:102DB000B5BA099400000000000000000000000007
:102DC000B5BAED91B5BAFE2FFF73B5BAE078E066FB
:102DD000B5BA0994000000000000000000000000E7
:102DE000B5BAED91B5BAFE2FFF73B5BAE078E067DA
:102DF000B5BA0994000000000000000000000000C7
:102E0000B5BAED91B5BAFE2FFF73B5BAE078E060C0
:102E1000B5BA0994000000000000000000000000A6
:102E2000B5BAED91B5BAFE2FFF73B5BAE078E0619F
:102E3000B5BA099400000000000000000000000086
:102E4000B5BAED91B5BAFE2FFF73B5BAE078E0627E
:102E5000B5BA099400000000000000000000000066
:102E6000B5BAED91B5BAFE2FFF73B5BAE078E0635D
:102E7000B5BA099400000000000000000000000046
:102E8000B5BAED91B5BAFE2FFF73B5BAE078E0643C
:102E9000B5BA099400000000000000000000000026
:102EA000B5BAED91A5BAFE2FFF73B5BAE078E0652B
:102EB000B5BA099400000000000000000000000006
:102EC000B5BAED91A5BAFE2FFF73B5BAE078E0660A
:102ED000B5BA0994000000000000000000000000E6
:102EE000B5BAED91B5BAFE2FFF73B5BAE078E067D9
:102EF000B5BA0994000000000000000000000000C6
:102F0000B5BAED91B5BAFE2FFF73B5BAE078E060BF
:102F1000B5BA0994000000000000000000000000A5
:102F2000B5BAED91B5BAFE2FFF73A5BAE078E061AE
:102F3000B5BA099400000000000000000000000085
:102F4000B5BAED91B5BAFE2FFF73A5BAE078E0628D
:102F5000B5BA099400000000000000000000000065
:102F6000B5BAED91A5BAFE2FFF73B5BAE078E0636C
:102F7000B5BA099400000000000000000000000045
:102F8000B5BAED91A5BAFE2FFF73B5BAE078E0644B
:102F9000B5BA099400000000000000000000000025
:102FA000A5BAED91B5BAFE2FFF73B5BAE078E0652A
:102FB000B5BA099400000000000000000000000005
:102FC000A5BAED91B5BAFE2FFF73B5BAE078E06609
:102FD000B5BA0994000000000000000000000000E5
:102FE000B5BAED91B5BAFE2FFF73B5BAE078E067D8
:102FF000B5BA0994000000000000000000000000C5
:10300000B5BAED91B5BAFE2FFF73B5BAE078E060BE
:10301000B5BA0994000000000000000000000000A4
:10302000B5BAED91A5BAFE2FFF73B5BAE078E061AD
:10303000B5BA099400000000000000000000000084
:10304000A5BAED91B5BAFE2FFF73A5BAE078E0629C
:10305000B5BA099400000000000000000000000064
:10306000A5BAED91B5BAFE2FFF73A5BAE078E0637B
:10307000B5BA099400000000000000000000000044
:10308000A5BAED91B5BAFE2FFF73A5BAE078E0645A
:10309000B5BA099400000000000000000000000024
:1030A000A5BAED91B5BAFE2FFF73A5BAE078E06539
:1030B000B5BA099400000000000000000000000004
:1030C000B5BAED91A5BAFE2FFF73B5BAE078E06608
:1030D000B5BA0994000000000000000000000000E4
:1030E000B5BAED91B5BAFE2FFF73B5BAE078E067D7
:1030F000B5BA0994000000000000000000000000C4
:10310000B5BAED91B5BAFE2FFF73B5BAE078E060BD
:10311000B5BA0994000000000000000000000000A3
:10312000B5BAED91A5BAFE2FFF73B5BAE078E061AC
:10313000B5BA099400000000000000000000000083
:10314000A5BAED91A5BAFE2FFF73B5BAE078E0629B
:10315000B5BA099400000000000000000000000063
:10316000B5BAED91A5BAFE2FFF73B5BAE078E0636A
:10317000B5BA099400000000000000000000000043
:10318000B5BAED91A5BAFE2FFF73B5BAE078E06449
:10319000B5BA099400000000000000000000000023
:1031A000B5BAED91A5BAFE2FFF73B5BAE078E06528
:1031B000B5BA099400000000000000000000000003
:1031C000A5BAED91A5BAFE2FFF73A5BAE078E06627
:1031D000B5BA0994000000000000000000000000E3
:1031E000B5BAED91B5BAFE2FFF73B5BAE078E067D6
:1031F000B5BA0994000000000000000000000000C3
:10320000B5BAED91B5BAFE2FFF73B5BAE078E060BC
:10321000B5BA0994000000000000000000000000A2
:10322000A5BAED91A5BAFE2FFF73B5BAE078E061BB
:10323000B5BA099400000000000000000000000082
:10324000B5BAED91B5BAFE2FFF73A5BAE078E0628A
:10325000B5BA099400000000000000000000000062
:10326000B5BAED91B5BAFE2FFF73A5BAE078E06369
:10327000B5BA099400000000000000000000000042
:10328000B5BAED91A5BAFE2FFF73B5BAE078E06448
:10329000B5BA099400000000000000000000000022
:1032A000A5BAED91B5BAFE2FFF73B5BAE078E06527
:1032B000B5BA099400000000000000000000000002
:1032C000A5BAED91A5BAFE2FFF73A5BAE078E06626
:1032D000B5BA0994000000000000000000000000E2
:1032E000B5BAED91B5BAFE2FFF73B5BAE078E067D5
:1032F000B5BA0994000000000000000000000000C2
:10330000B5BAED91B5BAFE2FFF73B5BAE078E060BB
:10331000B5BA0994000000000000000000000000A1
:10332000A5BAED91A5BAFE2FFF73B5BAE078E061BA
:10333000B5BA099400000000000000000000000081
:10334000B5BAED91B5BAFE2FFF73A5BAE078E06289
:10335000B5BA099400000000000000000000000061
:10336000B5BAED91A5BAFE2FFF73B5BAE078E06368
:10337000B5BA099400000000000000000000000041
:10338000B5BAED91B5BAFE2FFF73A5BAE078E06447
:10339000B5BA099400000000000000000000000021
:1033A000B5BAED91B5BAFE2FFF73A5BAE078E06526
:1033B000B5BA099400000000000000000000000001
:1033C000A5BAED91A5BAFE2FFF73B5BAE078E06615
:1033D000B5BA0994000000000000000000000000E1
:1033E000B5BAED91B5BAFE2FFF73B5BAE078E067D4
:1033F000B5BA0994000000000000000000000000C1
:10340000B5BAED91B5BAFE2FFF73B5BAE078E060BA
:10341000B5BA0994000000000000000000000000A0
:10342000A5BAED91B5BAFE2FFF73B5BAE078E061A9
:10343000B5BA099400000000000000000000000080
:10344000A5BAED91B5BAFE2FFF73A5BAE078E06298
:10345000B5BA099400000000000000000000000060
:10346000A5BAED91B5BAFE2FFF73A5BAE078E06377
:10347000B5BA099400000000000000000000000040
:10348000A5BAED91A5BAFE2FFF73A5BAE078E06466
:10349000B5BA099400000000000000000000000020
:1034A000B5BAED91B5BAFE2FFF73A5BAE078E06525
:1034B000B5BA099400000000000000000000000000
:1034C000B5BAED91B5BAFE2FFF73A5BAE078E06604
:1034D000B5BA0994000000000000000000000000E0
:1034E000B5BAED91B5BAFE2FFF73B5BAE078E067D3
:1034F000B5BA0994000000000000000000000000C0
:10350000B5BAED91B5BAFE2FFF73B5BAE078E060B9
:10351000B5BA09940000000000000000000000009F
:10352000A5BAED91A5BAFE2FFF73A5BAE078E061C8
:10353000B5BA09940000000000000000000000007F
:10354000A5BAED91B5BAFE2FFF73B5BAE078E06287
:10355000B5BA09940000000000000000000000005F
:10356000A5BAED91A5BAFE2FFF73B5BAE078E06376
:10357000B5BA09940000000000000000000000003F
:10358000B5BAED91B5BAFE2FFF73A5BAE078E06445
:10359000B5BA09940000000000000000000000001F
:1035A000B5BAED91B5BAFE2FFF73A5BAE078E06524
:1035B000B5BA0994000000000000000000000000FF
:1035C000A5BAED91A5BAFE2FFF73B5BAE078E06613
:1035D000B5BA0994000000000000000000000000DF
:1035E000B5BAED91B5BAFE2FFF73B5BAE078E067D2
:1035F000B5BA0994000000000000000000000000BF
:10360000B5BAED91B5BAFE2FFF73B5BAE078E060B8
:10361000B5BA09940000000000000000000000009E
:10362000B5BAED91A5BAFE2FFF73B5BAE078E061A7
:10363000B5BA09940000000000000000000000007E
:10364000A5BAED91B5BAFE2FFF73B5BAE078E06286
:10365000B5BA09940000000000000000000000005E
:10366000A5BAED91A5BAFE2FFF73B5BAE078E06375
:10367000B5BA09940000000000000000000000003E
:10368000A5BAED91B5BAFE2FFF73A5BAE078E06454
:10369000B5BA09940000000000000000000000001E
:1036A000A5BAED91B5BAFE2FFF73A5BAE078E06533
:1036B000B5BA0994000000000000000000000000FE
:1036C000B5BAED91A5BAFE2FFF73B5BAE078E06602
:1036D000B5BA0994000000000000000000000000DE
:1036E000B5BAED91B5BAFE2FFF73B5BAE078E067D1
:1036F000B5BA0994000000000000000000000000BE
:10370000B5BAED91B5BAFE2FFF73B5BAE078E060B7
:10371000B5BA09940000000000000000000000009D
:10372000A5BAED91A5BAFE2FFF73A5BAE078E061C6
:10373000B5BA09940000000000000000000000007D
:10374000B5BAED91B5BAFE2FFF73A5BAE078E06285
:10375000B5BA09940000000000000000000000005D
:10376000B5BAED91B5BAFE2FFF73A5BAE078E06364
:10377000B5BA09940000000000000000000000003D
:10378000B5BAED91A5BAFE2FFF73B5BAE078E06443
:10379000B5BA09940000000000000000000000001D
:1037A000A5BAED91B5BAFE2FFF73B5BAE078E06522
:1037B000B5BA0994000000000000000000000000FD
:1037C000A5BAED91B5BAFE2FFF73B5BAE078E06601
:1037D000B5BA0994000000000000000000000000DD
:1037E000B5BAED91B5BAFE2FFF73B5BAE078E067D0
:1037F000B5BA0994000000000000000000000000BD
:10380000B5BAED91B5BAFE2FFF73B5BAE078E060B6
:10381000B5BA09940000000000000000000000009C
:10382000B5BAED91A5BAFE2FFF73B5BAE078E061A5
:10383000B5BA09940000000000000000000000007C
:10384000A5BAED91B5BAFE2FFF73A5BAE078E06294
:10385000B5BA09940000000000000000000000005C
:10386000B5BAED91A5BAFE2FFF73B5BAE078E06363
:10387000B5BA09940000000000000000000000003C
:10388000A5BAED91B5BAFE2FFF73A5BAE078E06452
:10389000B5BA09940000000000000000000000001C
:1038A000A5BAED91B5BAFE2FFF73A5BAE078E06531
:1038B000B5BA0994000000000000000000000000FC
:1038C000B5BAED91A5BAFE2FFF73B5BAE078E06600
:1038D000B5BA0994000000000000000000000000DC
:1038E000B5BAED91B5BAFE2FFF73B5BAE078E067CF
:1038F000B5BA0994000000000000000000000000BC
:10390000B5BAED91B5BAFE2FFF73B5BAE078E060B5
:10391000B5BA09940000000000000000000000009B
:10392000B5BAED91A5BAFE2FFF73B5BAE078E061A4
:10393000B5BA09940000000000000000000000007B
:10394000A5BAED91B5BAFE2FFF73A5BAE078E06293
:10395000B5BA09940000000000000000000000005B
:10396000A5BAED91B5BAFE2FFF73A5BAE078E06372
:10397000B5BA09940000000000000000000000003B
:10398000B5BAED91A5BAFE2FFF73A5BAE078E06451
:10399000B5BA09940000000000000000000000001B
:1039A000B5BAED91B5BAFE2FFF73A5BAE078E06520
:1039B000B5BA0994000000000000000000000000FB
:1039C000B5BAED91A5BAFE2FFF73B5BAE078E066FF
:1039D000B5BA0994000000000000000000000000DB
:1039E000B5BAED91B5BAFE2FFF73B5BAE078E067CE
:1039F000B5BA0994000000000000000000000000BB
:103A0000B5BAED91B5BAFE2FFF73B5BAE078E060B4
:103A1000B5BA09940000000000000000000000009A
:103A2000B5BAED91B5BAFE2FFF73B5BAE078E06193
:103A3000B5BA09940000000000000000000000007A
:103A4000B5BAED91A5BAFE2FFF73B5BAE078E06282
:103A5000B5BA09940000000000000000000000005A
:103A6000B5BAED91A5BAFE2FFF73B5BAE078E06361
:103A7000B5BA09940000000000000000000000003A
:103A8000B5BAED91B5BAFE2FFF73B5BAE078E06430
:103A9000B5BA09940000000000000000000000001A
:103AA000B5BAED91A5BAFE2FFF73B5BAE078E0651F
:103AB000B5BA0994000000000000000000000000FA
:103AC000B5BAED91A5BAFE2FFF73B5BAE078E066FE
:103AD000B5BA0994000000000000000000000000DA
:103AE000B5BAED91B5BAFE2FFF73B5BAE078E067CD
:103AF000B5BA0994000000000000000000000000BA
:103B0000B5BAED91B5BAFE2FFF73B5BAE078E060B3
:103B1000B5BA099400000000000000000000000099
:103B2000B5BAED91B5BAFE2FFF73B5BAE078E06192
:103B3000B5BA099400000000000000000000000079
:103B4000B5BAED91A5BAFE2FFF73B5BAE078E06281
:103B5000B5BA099400000000000000000000000059
:103B6000B5BAED91A5BAFE2FFF73B5BAE078E06360
:103B7000B5BA099400000000000000000000000039
:103B8000B5BAED91B5BAFE2FFF73B5BAE078E0642F
:103B9000B5BA099400000000000000000000000019
:103BA000B5BAED91A5BAFE2FFF73B5BAE078E0651E
:103BB000B5BA0994000000000000000000000000F9
:103BC000B5BAED91A5BAFE2FFF73B5BAE078E066FD
:103BD000B5BA0994000000000000000000000000D9
:103BE000A5BAED91B5BAFE2FFF73B5BAE078E067DC
:103BF000B5BA0994000000000000000000000000B9
:103C0000B5BAED91B5BAFE2FFF73B5BAE078E060B2
:103C1000B5BA099400000000000000000000000098
:103C2000B5BAED91B5BAFE2FFF73B5BAE078E06191
:103C3000B5BA099400000000000000000000000078
:103C4000B5BAED91B5BAFE2FFF73A5BAE078E06280
:103C5000B5BA099400000000000000000000000058
:103C6000B5BAED91A5BAFE2FFF73B5BAE078E0635F
:103C7000B5BA099400000000000000000000000038
:103C8000A5BAED91B5BAFE2FFF73B5BAE078E0643E
:103C9000B5BA099400000000000000000000000018
:103CA000B5BAED91A5BAFE2FFF73B5BAE078E0651D
:103CB000B5BA0994000000000000000000000000F8
:103CC000B5BAED91B5BAFE2FFF73A5BAE078E066FC
:103CD000B5BA0994000000000000000000000000D8
:103CE000B5BAED91B5BAFE2FFF73B5BAE078E067CB
:103CF000B5BA0994000000000000000000000000B8
:103D0000B5BAED91B5BAFE2FFF73B5BAE078E060B1
:103D1000B5BA099400000000000000000000000097
:103D2000B5BAED91B5BAFE2FFF73B5BAE078E06190
:103D3000B5BA099400000000000000000000000077
:103D4000B5BAED91B5BAFE2FFF73B5BAE078E0626F
:103D5000B5BA099400000000000000000000000057
:103D6000A5BAED91A5BAFE2FFF73A5BAE078E0637E
:103D7000B5BA099400000000000000000000000037
:103D8000B5BAED91B5BAFE2FFF73B5BAE078E0642D
:103D9000B5BA099400000000000000000000000017
:103DA000A5BAED91A5BAFE2FFF73A5BAE078E0653C
:103DB000B5BA0994000000000000000000000000F7
:103DC000B5BAED91B5BAFE2FFF73B5BAE078E066EB
:103DD000B5BA0994000000000000000000000000D7
:103DE000B5BAED91B5BAFE2FFF73B5BAE078E067CA
:103DF000B5BA0994000000000000000000000000B7
:103E0000B5BAED91B5BAFE2FFF73B5BAE078E060B0
:103E1000B5BA099400000000000000000000000096
:103E2000B5BAED91B5BAFE2FFF73B5BAE078E0618F
:103E3000B5BA099400000000000000000000000076
:103E4000A5BAED91B5BAFE2FFF73B5BAE078E0627E
:103E5000B5BA099400000000000000000000000056
:103E6000B5BAED91A5BAFE2FFF73B5BAE078E0635D
:103E7000B5BA099400000000000000000000000036
:103E8000B5BAED91B5BAFE2FFF73A5BAE078E0643C
:103E9000B5BA099400000000000000000000000016
:103EA000B5BAED91A5BAFE2FFF73B5BAE078E0651B
:103EB000B5BA0994000000000000000000000000F6
:103EC000A5BAED91B5BAFE2FFF73B5BAE078E066FA
:103ED000B5BA0994000000000000000000000000D6
:103EE000B5BAED91B5BAFE2FFF73B5BAE078E067C9
:103EF000B5BA0994000000000000000000000000B6
:103F0000B5BAED91B5BAFE2FFF73B5BAE078E060AF
:103F1000B5BA099400000000000000000000000095
:103F2000A5BAED91A5BAFE2FFF73B5BAE078E061AE
:103F3000B5BA099400000000000000000000000075
:103F4000B5BAED91B5BAFE2FFF73A5BAE078E0627D
:103F5000B5BA099400000000000000000000000055
:103F6000B5BAED91A5BAFE2FFF73B5BAE078E0635C
:103F7000B5BA099400000000000000000000000035
:103F8000B5BAED91A5BAFE2FFF73B5BAE078E0643B
:103F9000B5BA099400000000000000000000000015
:103FA000B5BAED91B5BAFE2FFF73B5BAE078E0650A
:103FB000B5BA0994000000000000000000000000F5
:103FC000B5BAED91A5BAFE2FFF73B5BAE078E066F9
:103FD000B5BA0994000000000000000000000000D5
:103FE000B5BAED91B5BAFE2FFF73B5BAE078E067C8
:103FF000B5BA0994000000000000000000000000B5
:10400000B5BAED91B5BAFE2FFF73B5BAE078E060AE
:10401000B5BA099400000000000000000000000094
:10402000B5BAED91A5BAFE2FFF73B5BAE078E0619D
:10403000B5BA099400000000000000000000000074
:10404000A5BAED91B5BAFE2FFF73A5BAE078E0628C
:10405000B5BA099400000000000000000000000054
:10406000A5BAED91A5BAFE2FFF73A5BAE078E0637B
:10407000B5BA099400000000000000000000000034
:10408000A5BAED91A5BAFE2FFF73A5BAE078E0645A
:10409000B5BA099400000000000000000000000014
:1040A000A5BAED91B5BAFE2FFF73B5BAE078E06519
:1040B000B5BA0994000000000000000000000000F4
:1040C000B5BAED91A5BAFE2FFF73A5BAE078E06608
:1040D000B5BA0994000000000000000000000000D4
:1040E000B5BAED91B5BAFE2FFF73B5BAE078E067C7
:1040F000B5BA0994000000000000000000000000B4
:10410000B5BAED91B5BAFE2FFF73B5BAE078E060AD
:10411000B5BA099400000000000000000000000093
:10412000B5BAED91A5BAFE2FFF73B5BAE078E0619C
:10413000B5BA099400000000000000000000000073
:10414000A5BAED91B5BAFE2FFF73A5BAE078E0628B
:10415000B5BA099400000000000000000000000053
:10416000A5BAED91B5BAFE2FFF73A5BAE078E0636A
:10417000B5BA099400000000000000000000000033
:10418000A5BAED91A5BAFE2FFF73A5BAE078E06459
:10419000B5BA099400000000000000000000000013
:1041A000A5BAED91B5BAFE2FFF73A5BAE078E06528
:1041B000B5BA0994000000000000000000000000F3
:1041C000A5BAED91B5BAFE2FFF73A5BAE078E06607
:1041D000B5BA0994000000000000000000000000D3
:1041E000B5BAED91B5BAFE2FFF73B5BAE078E067C6
:1041F000B5BA0994000000000000000000000000B3
:10420000B5BAED91B5BAFE2FFF73B5BAE078E060AC
:10421000B5BA099400000000000000000000000092
:10422000A5BAED91A5BAFE2FFF73B5BAE078E061AB
:10423000B5BA099400000000000000000000000072
:10424000A5BAED91B5BAFE2FFF73A5BAE078E0628A
:10425000B5BA099400000000000000000000000052
:10426000A5BAED91A5BAFE2FFF73B5BAE078E06369
:10427000B5BA099400000000000000000000000032
:10428000A5BAED91B5BAFE2FFF73A5BAE078E06448
:10429000B5BA099400000000000000000000000012
:1042A000A5BAED91B5BAFE2FFF73A5BAE078E06527
:1042B000B5BA0994000000000000000000000000F2
:1042C000A5BAED91A5BAFE2FFF73B5BAE078E06606
:1042D000B5BA0994000000000000000000000000D2
:1042E000B5BAED91B5BAFE2FFF73B5BAE078E067C5
:1042F000B5BA0994000000000000000000000000B2
:10430000B5BAED91B5BAFE2FFF73B5BAE078E060AB
:10431000B5BA099400000000000000000000000091
:10432000B5BAED91A5BAFE2FFF73A5BAE078E061AA
:10433000B5BA099400000000000000000000000071
:10434000A5BAED91B5BAFE2FFF73B5BAE078E06279
:10435000B5BA099400000000000000000000000051
:10436000A5BAED91B5BAFE2FFF73B5BAE078E06358
:10437000B5BA099400000000000000000000000031
:10438000A5BAED91B5BAFE2FFF73B5BAE078E06437
:10439000B5BA099400000000000000000000000011
:1043A000A5BAED91B5BAFE2FFF73B5BAE078E06516
:1043B000B5BA0994000000000000000000000000F1
:1043C000B5BAED91A5BAFE2FFF73A5BAE078E06605
:1043D000B5BA0994000000000000000000000000D1
:1043E000B5BAED91B5BAFE2FFF73B5BAE078E067C4
:1043F000B5BA0994000000000000000000000000B1
:10440000B5BAED91B5BAFE2FFF73B5BAE078E060AA
:10441000B5BA099400000000000000000000000090
:10442000A5BAED91A5BAFE2FFF73B5BAE078E061A9
:10443000B5BA099400000000000000000000000070
:10444000A5BAED91B5BAFE2FFF73A5BAE078E06288
:10445000B5BA099400000000000000000000000050
:10446000A5BAED91B5BAFE2FFF73A5BAE078E06367
:10447000B5BA099400000000000000000000000030
:10448000A5BAED91B5BAFE2FFF73A5BAE078E06446
:10449000B5BA099400000000000000000000000010
:1044A000A5BAED91B5BAFE2FFF73A5BAE078E06525
:1044B000B5BA0994000000000000000000000000F0
:1044C000A5BAED91A5BAFE2FFF73B5BAE078E06604
:1044D000B5BA0994000000000000000000000000D0
:1044E000B5BAED91B5BAFE2FFF73B5BAE078E067C3
:1044F000B5BA0994000000000000000000000000B0
:10450000B5BAED91B5BAFE2FFF73B5BAE078E060A9
:10451000B5BA09940000000000000000000000008F
:10452000A5BAED91A5BAFE2FFF73A5BAE078E061B8
:10453000B5BA09940000000000000000000000006F
:10454000A5BAED91B5BAFE2FFF73B5BAE078E06277
:10455000B5BA09940000000000000000000000004F
:10456000A5BAED91A5BAFE2FFF73B5BAE078E06366
:10457000B5BA09940000000000000000000000002F
:10458000A5BAED91B5BAFE2FFF73B5BAE078E06435
:10459000B5BA09940000000000000000000000000F
:1045A000A5BAED91B5BAFE2FFF73B5BAE078E06514
:1045B000B5BA0994000000000000000000000000EF
:1045C000A5BAED91A5BAFE2FFF73A5BAE078E06613
:1045D000B5BA0994000000000000000000000000CF
:1045E000B5BAED91B5BAFE2FFF73B5BAE078E067C2
:1045F000B5BA0994000000000000000000000000AF
:10460000B5BAED91B5BAFE2FFF73B5BAE078E060A8
:10461000B5BA09940000000000000000000000008E
:10462000A5BAED91A5BAFE2FFF73A5BAE078E061B7
:10463000B5BA09940000000000000000000000006E
:10464000A5BAED91B5BAFE2FFF73B5BAE078E06276
:10465000B5BA09940000000000000000000000004E
:10466000A5BAED91B5BAFE2FFF73B5BAE078E06355
:10467000B5BA09940000000000000000000000002E
:10468000A5BAED91A5BAFE2FFF73B5BAE078E06444
:10469000B5BA09940000000000000000000000000E
:1046A000A5BAED91B5BAFE2FFF73B5BAE078E06513
:1046B000B5BA0994000000000000000000000000EE
:1046C000A5BAED91B5BAFE2FFF73B5BAE078E066F2
:1046D000B5BA0994000000000000000000000000CE
:1046E000B5BAED91B5BAFE2FFF73B5BAE078E067C1
:1046F000B5BA0994000000000000000000000000AE
:10470000B5BAED91B5BAFE2FFF73B5BAE078E060A7
:10471000B5BA09940000000000000000000000008D
:10472000B5BAED91A5BAFE2FFF73A5BAE078E061A6
:10473000B5BA09940000000000000000000000006D
:10474000A5BAED91B5BAFE2FFF73B5BAE078E06275
:10475000B5BA09940000000000000000000000004D
:10476000A5BAED91B5BAFE2FFF73B5BAE078E06354
:10477000B5BA09940000000000000000000000002D
:10478000A5BAED91B5BAFE2FFF73A5BAE078E06443
:10479000B5BA09940000000000000000000000000D
:1047A000A5BAED91B5BAFE2FFF73A5BAE078E06522
:1047B000B5BA0994000000000000000000000000ED
:1047C000B5BAED91A5BAFE2FFF73A5BAE078E06601
:1047D000B5BA0994000000000000000000000000CD
:1047E000B5BAED91B5BAFE2FFF73B5BAE078E067C0
:1047F000B5BA0994000000000000000000000000AD
:10480000B5BAED91B5BAFE2FFF73B5BAE078E060A6
:10481000B5BA09940000000000000000000000008C
:10482000A5BAED91B5BAFE2FFF73A5BAE078E061A5
:10483000B5BA09940000000000000000000000006C
:10484000A5BAED91B5BAFE2FFF73A5BAE078E06284
:10485000B5BA09940000000000000000000000004C
:10486000A5BAED91A5BAFE2FFF73A5BAE078E06373
:10487000B5BA09940000000000000000000000002C
:10488000A5BAED91B5BAFE2FFF73A5BAE078E06442
:10489000B5BA09940000000000000000000000000C
:1048A000A5BAED91B5BAFE2FFF73A5BAE078E06521
:1048B000B5BA0994000000000000000000000000EC
:1048C000A5BAED91B5BAFE2FFF73A5BAE078E06600
:1048D000B5BA0994000000000000000000000000CC
:1048E000B5BAED91B5BAFE2FFF73B5BAE078E067BF
:1048F000B5BA0994000000000000000000000000AC
:10490000B5BAED91B5BAFE2FFF73B5BAE078E060A5
:10491000B5BA09940000000000000000000000008B
:10492000A5BAED91A5BAFE2FFF73A5BAE078E061B4
:10493000B5BA09940000000000000000000000006B
:10494000B5BAED91A5BAFE2FFF73B5BAE078E06273
:10495000B5BA09940000000000000000000000004B
:10496000B5BAED91A5BAFE2FFF73B5BAE078E06352
:10497000B5BA09940000000000000000000000002B
:10498000B5BAED91A5BAFE2FFF73B5BAE078E06431
:10499000B5BA09940000000000000000000000000B
:1049A000B5BAED91A5BAFE2FFF73B5BAE078E06510
:1049B000B5BA0994000000000000000000000000EB
:1049C000A5BAED91A5BAFE2FFF73A5BAE078E0660F
:1049D000B5BA0994000000000000000000000000CB
:1049E000B5BAED91B5BAFE2FFF73B5BAE078E067BE
:1049F000B5BA0994000000000000000000000000AB
:104A0000B5BAED91B5BAFE2FFF73B5BAE078E060A4
:104A1000B5BA09940000000000000000000000008A
:104A2000A5BAED91A5BAFE2FFF73A5BAE078E061B3
:104A3000B5BA09940000000000000000000000006A
:104A4000B5BAED91A5BAFE2FFF73B5BAE078E06272
:104A5000B5BA09940000000000000000000000004A
:104A6000B5BAED91A5BAFE2FFF73B5BAE078E06351
:104A7000B5BA09940000000000000000000000002A
:104A8000B5BAED91A5BAFE2FFF73B5BAE078E06430
:104A9000B5BA09940000000000000000000000000A
:104AA000B5BAED91A5BAFE2FFF73B5BAE078E0650F
:104AB000B5BA0994000000000000000000000000EA
:104AC000A5BAED91B5BAFE2FFF73B5BAE078E066EE
:104AD000B5BA0994000000000000000000000000CA
:104AE000B5BAED91B5BAFE2FFF73B5BAE078E067BD
:104AF000B5BA0994000000000000000000000000AA
:104B0000B5BAED91B5BAFE2FFF73B5BAE078E060A3
:104B1000B5BA099400000000000000000000000089
:104B2000A5BAED91B5BAFE2FFF73A5BAE078E061A2
:104B3000B5BA099400000000000000000000000069
:104B4000A5BAED91B5BAFE2FFF73A5BAE078E06281
:104B5000B5BA099400000000000000000000000049
:104B6000A5BAED91A5BAFE2FFF73B5BAE078E06360
:104B7000B5BA099400000000000000000000000029
:104B8000A5BAED91A5BAFE2FFF73B5BAE078E0643F
:104B9000B5BA099400000000000000000000000009
:104BA000A5BAED91B5BAFE2FFF73A5BAE078E0651E
:104BB000B5BA0994000000000000000000000000E9
:104BC000A5BAED91B5BAFE2FFF73A5BAE078E066FD
:104BD000B5BA0994000000000000000000000000C9
:104BE000B5BAED91B5BAFE2FFF73B5BAE078E067BC
:104BF000B5BA0994000000000000000000000000A9
:104C0000B5BAED91B5BAFE2FFF73B5BAE078E060A2
:104C1000B5BA099400000000000000000000000088
:104C2000A5BAED91B5BAFE2FFF73B5BAE078E06191
:104C3000B5BA099400000000000000000000000068
:104C4000A5BAED91B5BAFE2FFF73B5BAE078E06270
:104C5000B5BA099400000000000000000000000048
:104C6000A5BAED91B5BAFE2FFF73B5BAE078E0634F
:104C7000B5BA099400000000000000000000000028
:104C8000A5BAED91B5BAFE2FFF73B5BAE078E0642E
:104C9000B5BA099400000000000000000000000008
:104CA000A5BAED91B5BAFE2FFF73B5BAE078E0650D
:104CB000B5BA0994000000000000000000000000E8
:104CC000A5BAED91A5BAFE2FFF73A5BAE078E0660C
:104CD000B5BA0994000000000000000000000000C8
:104CE000B5BAED91B5BAFE2FFF73B5BAE078E067BB
:104CF000B5BA0994000000000000000000000000A8
:104D0000B5BAED91B5BAFE2FFF73B5BAE078E060A1
:104D1000B5BA099400000000000000000000000087
:104D2000A5BAED91B5BAFE2FFF73A5BAE078E061A0
:104D3000B5BA099400000000000000000000000067
:104D4000A5BAED91A5BAFE2FFF73A5BAE078E0628F
:104D5000B5BA099400000000000000000000000047
:104D6000A5BAED91A5BAFE2FFF73A5BAE078E0636E
:104D7000B5BA099400000000000000000000000027
:104D8000A5BAED91B5BAFE2FFF73A5BAE078E0643D
:104D9000B5BA099400000000000000000000000007
:104DA000A5BAED91B5BAFE2FFF73A5BAE078E0651C
:104DB000B5BA0994000000000000000000000000E7
:104DC000A5BAED91B5BAFE2FFF73A5BAE078E066FB
:104DD000B5BA0994000000000000000000000000C7
:104DE000B5BAED91B5BAFE2FFF73B5BAE078E067BA
:104DF000B5BA0994000000000000000000000000A7
:104E0000B5BAED91B5BAFE2FFF73B5BAE078E060A0
:104E1000B5BA099400000000000000000000000086
:104E2000A5BAED91B5BAFE2FFF73A5BAE078E0619F
:104E3000B5BA099400000000000000000000000066
:104E4000A5BAED91A5BAFE2FFF73A5BAE078E0628E
:104E5000B5BA099400000000000000000000000046
:104E6000A5BAED91A5BAFE2FFF73A5BAE078E0636D
:104E7000B5BA099400000000000000000000000026
:104E8000A5BAED91A5BAFE2FFF73A5BAE078E0644C
:104E9000B5BA099400000000000000000000000006
:104EA000A5BAED91A5BAFE2FFF73A5BAE078E0652B
:104EB000B5BA0994000000000000000000000000E6
:104EC000A5BAED91B5BAFE2FFF73A5BAE078E066FA
:104ED000B5BA0994000000000000000000000000C6
:104EE000B5BAED91B5BAFE2FFF73B5BAE078E067B9
:104EF000B5BA0994000000000000000000000000A6
:104F0000B5BAED91B5BAFE2FFF73B5BAE078E0609F
:104F1000B5BA099400000000000000000000000085
:104F2000B5BAED91A5BAFE2FFF73B5BAE078E0618E
:104F3000B5BA099400000000000000000000000065
:104F4000A5BAED91B5BAFE2FFF73A5BAE078E0627D
:104F5000B5BA099400000000000000000000000045
:104F6000A5BAED91B5BAFE2FFF73A5BAE078E0635C
:104F7000B5BA099400000000000000000000000025
:104F8000A5BAED91B5BAFE2FFF73A5BAE078E0643B
:104F9000B5BA099400000000000000000000000005
:104FA000A5BAED91B5BAFE2FFF73A5BAE078E0651A
:104FB000B5BA0994000000000000000000000000E5
:104FC000B5BAED91A5BAFE2FFF73B5BAE078E066E9
:104FD000B5BA0994000000000000000000000000C5
:104FE000B5BAED91B5BAFE2FFF73B5BAE078E067B8
:104FF000B5BA0994000000000000000000000000A5
:10500000B5BAED91B5BAFE2FFF73B5BAE078E0609E
:10501000B5BA099400000000000000000000000084
:10502000A5BAED91A5BAFE2FFF73B5BAE078E0619D
:10503000B5BA099400000000000000000000000064
:10504000A5BAED91B5BAFE2FFF73A5BAE078E0627C
:10505000B5BA099400000000000000000000000044
:10506000A5BAED91B5BAFE2FFF73A5BAE078E0635B
:10507000B5BA099400000000000000000000000024
:10508000A5BAED91A5BAFE2FFF73B5BAE078E0643A
:10509000B5BA099400000000000000000000000004
:1050A000A5BAED91B5BAFE2FFF73B5BAE078E06509
:1050B000B5BA0994000000000000000000000000E4
:1050C000A5BAED91B5BAFE2FFF73B5BAE078E066E8
:1050D000B5BA0994000000000000000000000000C4
:1050E000B5BAED91B5BAFE2FFF73B5BAE078E067B7
:1050F000B5BA0994000000000000000000000000A4
:10510000B5BAED91B5BAFE2FFF73B5BAE078E0609D
:10511000B5BA099400000000000000000000000083
:10512000B5BAED91A5BAFE2FFF73B5BAE078E0618C
:10513000B5BA099400000000000000000000000063
:10514000A5BAED91B5BAFE2FFF73A5BAE078E0627B
:10515000B5BA099400000000000000000000000043
:10516000A5BAED91B5BAFE2FFF73A5BAE078E0635A
:10517000B5BA099400000000000000000000000023
:10518000A5BAED91B5BAFE2FFF73A5BAE078E06439
:10519000B5BA099400000000000000000000000003
:1051A000A5BAED91A5BAFE2FFF73A5BAE078E06528
:1051B000B5BA0994000000000000000000000000E3
:1051C000B5BAED91A5BAFE2FFF73A5BAE078E066F7
:1051D000B5BA0994000000000000000000000000C3
:1051E000B5BAED91B5BAFE2FFF73B5BAE078E067B6
:1051F000B5BA0994000000000000000000000000A3
:10520000B5BAED91B5BAFE2FFF73B5BAE078E0609C
:10521000B5BA099400000000000000000000000082
:10522000A5BAED91A5BAFE2FFF73B5BAE078E0619B
:10523000B5BA099400000000000000000000000062
:10524000A5BAED91B5BAFE2FFF73A5BAE078E0627A
:10525000B5BA099400000000000000000000000042
:10526000A5BAED91B5BAFE2FFF73A5BAE078E06359
:10527000B5BA099400000000000000000000000022
:10528000A5BAED91A5BAFE2FFF73B5BAE078E06438
:10529000B5BA099400000000000000000000000002
:1052A000A5BAED91B5BAFE2FFF73A5BAE078E06517
:1052B000B5BA0994000000000000000000000000E2
:1052C000A5BAED91B5BAFE2FFF73A5BAE078E066F6
:1052D000B5BA0994000000000000000000000000C2
:1052E000B5BAED91B5BAFE2FFF73B5BAE078E067B5
:1052F000B5BA0994000000000000000000000000A2
:10530000B5BAED91B5BAFE2FFF73B5BAE078E0609B
:10531000B5BA099400000000000000000000000081
:10532000B5BAED91A5BAFE2FFF73A5BAE078E0619A
:10533000B5BA099400000000000000000000000061
:10534000A5BAED91B5BAFE2FFF73B5BAE078E06269
:10535000B5BA099400000000000000000000000041
:10536000B5BAED91A5BAFE2FFF73B5BAE078E06348
:10537000B5BA099400000000000000000000000021
:10538000B5BAED91B5BAFE2FFF73A5BAE078E06427
:10539000B5BA099400000000000000000000000001
:1053A000B5BAED91B5BAFE2FFF73A5BAE078E06506
:1053B000B5BA0994000000000000000000000000E1
:1053C000A5BAED91A5BAFE2FFF73B5BAE078E066F5
:1053D000B5BA0994000000000000000000000000C1
:1053E000B5BAED91B5BAFE2FFF73B5BAE078E067B4
:1053F000B5BA0994000000000000000000000000A1
:10540000B5BAED91B5BAFE2FFF73B5BAE078E0609A
:10541000B5BA099400000000000000000000000080
:10542000A5BAED91A5BAFE2FFF73A5BAE078E061A9
:10543000B5BA099400000000000000000000000060
:10544000B5BAED91A5BAFE2FFF73B5BAE078E06268
:10545000B5BA099400000000000000000000000040
:10546000B5BAED91A5BAFE2FFF73B5BAE078E06347
:10547000B5BA099400000000000000000000000020
:10548000B5BAED91A5BAFE2FFF73B5BAE078E06426
:10549000B5BA099400000000000000000000000000
:1054A000B5BAED91A5BAFE2FFF73B5BAE078E06505
:1054B000B5BA0994000000000000000000000000E0
:1054C000B5BAED91A5BAFE2FFF73B5BAE078E066E4
:1054D000B5BA0994000000000000000000000000C0
:1054E000B5BAED91B5BAFE2FFF73B5BAE078E067B3
:1054F000B5BA0994000000000000000000000000A0
:10550000B5BAED91B5BAFE2FFF73B5BAE078E06099
:10551000B5BA09940000000000000000000000007F
:10552000A5BAED91B5BAFE2FFF73A5BAE078E06198
:10553000B5BA09940000000000000000000000005F
:10554000A5BAED91B5BAFE2FFF73A5BAE078E06277
:10555000B5BA09940000000000000000000000003F
:10556000A5BAED91B5BAFE2FFF73A5BAE078E06356
:10557000B5BA09940000000000000000000000001F
:10558000A5BAED91B5BAFE2FFF73A5BAE078E06435
:10559000B5BA0994000000000000000000000000FF
:1055A000A5BAED91B5BAFE2FFF73A5BAE078E06514
:1055B000B5BA0994000000000000000000000000DF
:1055C000B5BAED91A5BAFE2FFF73B5BAE078E066E3
:1055D000B5BA0994000000000000000000000000BF
:1055E000B5BAED91B5BAFE2FFF73B5BAE078E067B2
:1055F000B5BA09940000000000000000000000009F
:10560000B5BAED91B5BAFE2FFF73B5BAE078E06098
:10561000B5BA09940000000000000000000000007E
:10562000A5BAED91B5BAFE2FFF73A5BAE078E06197
:10563000B5BA09940000000000000000000000005E
:10564000A5BAED91B5BAFE2FFF73A5BAE078E06276
:10565000B5BA09940000000000000000000000003E
:10566000A5BAED91B5BAFE2FFF73A5BAE078E06355
:10567000B5BA09940000000000000000000000001E
:10568000A5BAED91B5BAFE2FFF73A5BAE078E06434
:10569000B5BA0994000000000000000000000000FE
:1056A000B5BAED91A5BAFE2FFF73B5BAE078E06503
:1056B000B5BA0994000000000000000000000000DE
:1056C000B5BAED91A5BAFE2FFF73B5BAE078E066E2
:1056D000B5BA0994000000000000000000000000BE
:1056E000B5BAED91B5BAFE2FFF73B5BAE078E067B1
:1056F000B5BA09940000000000000000000000009E
:10570000B5BAED91B5BAFE2FFF73B5BAE078E06097
:10571000B5BA09940000000000000000000000007D
:10572000A5BAED91B5BAFE2FFF73A5BAE078E06196
:10573000B5BA09940000000000000000000000005D
:10574000A5BAED91B5BAFE2FFF73A5BAE078E06275
:10575000B5BA09940000000000000000000000003D
:10576000A5BAED91B5BAFE2FFF73A5BAE078E06354
:10577000B5BA09940000000000000000000000001D
:10578000A5BAED91A5BAFE2FFF73A5BAE078E06443
:10579000B5BA0994000000000000000000000000FD
:1057A000A5BAED91A5BAFE2FFF73A5BAE078E06522
:1057B000B5BA0994000000000000000000000000DD
:1057C000A5BAED91B5BAFE2FFF73A5BAE078E066F1
:1057D000B5BA0994000000000000000000000000BD
:1057E000B5BAED91B5BAFE2FFF73B5BAE078E067B0
:1057F000B5BA09940000000000000000000000009D
:10580000B5BAED91B5BAFE2FFF73B5BAE078E06096
:10581000B5BA09940000000000000000000000007C
:10582000A5BAED91B5BAFE2FFF73A5BAE078E06195
:10583000B5BA09940000000000000000000000005C
:10584000A5BAED91B5BAFE2FFF73A5BAE078E06274
:10585000B5BA09940000000000000000000000003C
:10586000B5BAED91A5BAFE2FFF73B5BAE078E06343
:10587000B5BA09940000000000000000000000001C
:10588000B5BAED91A5BAFE2FFF73B5BAE078E06422
:10589000B5BA0994000000000000000000000000FC
:1058A000A5BAED91B5BAFE2FFF73A5BAE078E06511
:1058B000B5BA0994000000000000000000000000DC
:1058C000A5BAED91B5BAFE2FFF73A5BAE078E066F0
:1058D000B5BA0994000000000000000000000000BC
:1058E000B5BAED91B5BAFE2FFF73B5BAE078E067AF
:1058F000B5BA09940000000000000000000000009C
:10590000B5BAED91B5BAFE2FFF73B5BAE078E06095
:10591000B5BA09940000000000000000000000007B
:10592000A5BAED91B5BAFE2FFF73A5BAE078E06194
:10593000B5BA09940000000000000000000000005B
:10594000A5BAED91B5BAFE2FFF73A5BAE078E06273
:10595000B5BA09940000000000000000000000003B
:10596000A5BAED91B5BAFE2FFF73A5BAE078E06352
:10597000B5BA09940000000000000000000000001B
:10598000B5BAED91A5BAFE2FFF73B5BAE078E06421
:10599000B5BA0994000000000000000000000000FB
:1059A000B5BAED91A5BAFE2FFF73B5BAE078E06500
:1059B000B5BA0994000000000000000000000000DB
:1059C000B5BAED91A5BAFE2FFF73B5BAE078E066DF
:1059D000B5BA0994000000000000000000000000BB
:1059E000B5BAED91B5BAFE2FFF73B5BAE078E067AE
:1059F000B5BA09940000000000000000000000009B
:105A0000B5BAED91B5BAFE2FFF73B5BAE078E06094
:105A1000B5BA09940000000000000000000000007A
:105A2000A5BAED91A5BAFE2FFF73A5BAE078E061A3
:105A3000B5BA09940000000000000000000000005A
:105A4000B5BAED91B5BAFE2FFF73A5BAE078E06262
:105A5000B5BA09940000000000000000000000003A
:105A6000B5BAED91A5BAFE2FFF73B5BAE078E06341
:105A7000B5BA09940000000000000000000000001A
:105A8000B5BAED91A5BAFE2FFF73B5BAE078E06420
:105A9000B5BA0994000000000000000000000000FA
:105AA000A5BAED91B5BAFE2FFF73B5BAE078E065FF
:105AB000B5BA0994000000000000000000000000DA
:105AC000A5BAED91A5BAFE2FFF73A5BAE078E066FE
:105AD000B5BA0994000000000000000000000000BA
:105AE000B5BAED91B5BAFE2FFF73B5BAE078E067AD
:105AF000B5BA09940000000000000000000000009A
:105B0000B5BAED91B5BAFE2FFF73B5BAE078E06093
:105B1000B5BA099400000000000000000000000079
:105B2000B5BAED91A5BAFE2FFF73A5BAE078E06192
:105B3000B5BA099400000000000000000000000059
:105B4000B5BAED91A5BAFE2FFF73B5BAE078E06261
:105B5000B5BA099400000000000000000000000039
:105B6000B5BAED91A5BAFE2FFF73B5BAE078E06340
:105B7000B5BA099400000000000000000000000019
:105B8000B5BAED91A5BAFE2FFF73B5BAE078E0641F
:105B9000B5BA0994000000000000000000000000F9
:105BA000B5BAED91A5BAFE2FFF73B5BAE078E065FE
:105BB000B5BA0994000000000000000000000000D9
:105BC000B5BAED91A5BAFE2FFF73A5BAE078E066ED
:105BD000B5BA0994000000000000000000000000B9
:105BE000B5BAED91B5BAFE2FFF73B5BAE078E067AC
:105BF000B5BA099400000000000000000000000099
:105C0000B5BAED91B5BAFE2FFF73B5BAE078E06092
:105C1000B5BA099400000000000000000000000078
:105C2000A5BAED91B5BAFE2FFF73B5BAE078E06181
:105C3000B5BA099400000000000000000000000058
:105C4000A5BAED91B5BAFE2FFF73B5BAE078E06260
:105C5000B5BA099400000000000000000000000038
:105C6000B5BAED91A5BAFE2FFF73B5BAE078E0633F
:105C7000B5BA099400000000000000000000000018
:105C8000B5BAED91A5BAFE2FFF73B5BAE078E0641E
:105C9000B5BA0994000000000000000000000000F8
:105CA000B5BAED91B5BAFE2FFF73A5BAE078E065FD
:105CB000B5BA0994000000000000000000000000D8
:105CC000B5BAED91B5BAFE2FFF73A5BAE078E066DC
:105CD000B5BA0994000000000000000000000000B8
:105CE000B5BAED91B5BAFE2FFF73B5BAE078E067AB
:105CF000B5BA099400000000000000000000000098
:105D0000B5BAED91B5BAFE2FFF73B5BAE078E06091
:105D1000B5BA099400000000000000000000000077
:105D2000A5BAED91A5BAFE2FFF73B5BAE078E06190
:105D3000B5BA099400000000000000000000000057
:105D4000B5BAED91A5BAFE2FFF73B5BAE078E0625F
:105D5000B5BA099400000000000000000000000037
:105D6000B5BAED91A5BAFE2FFF73B5BAE078E0633E
:105D7000B5BA099400000000000000000000000017
:105D8000B5BAED91A5BAFE2FFF73B5BAE078E0641D
:105D9000B5BA0994000000000000000000000000F7
:105DA000B5BAED91A5BAFE2FFF73B5BAE078E065FC
:105DB000B5BA0994000000000000000000000000D7
:105DC000A5BAED91A5BAFE2FFF73B5BAE078E066EB
:105DD000B5BA0994000000000000000000000000B7
:105DE000B5BAED91B5BAFE2FFF73B5BAE078E067AA
:105DF000B5BA099400000000000000000000000097
:105E0000B5BAED91B5BAFE2FFF73B5BAE078E06090
:105E1000B5BA099400000000000000000000000076
:105E2000B5BAED91A5BAFE2FFF73B5BAE078E0617F
:105E3000B5BA099400000000000000000000000056
:105E4000A5BAED91B5BAFE2FFF73A5BAE078E0626E
:105E5000B5BA099400000000000000000000000036
:105E6000B5BAED91B5BAFE2FFF73B5BAE078E0632D
:105E7000B5BA099400000000000000000000000016
:105E8000B5BAED91B5BAFE2FFF73B5BAE078E0640C
:105E9000B5BA0994000000000000000000000000F6
:105EA000B5BAED91B5BAFE2FFF73B5BAE078E065EB
:105EB000B5BA0994000000000000000000000000D6
:105EC000B5BAED91B5BAFE2FFF73B5BAE078E066CA
:105ED000B5BA0994000000000000000000000000B6
:105EE000B5BAED91B5BAFE2FFF73B5BAE078E067A9
:105EF000B5BA099400000000000000000000000096
:105F0000B5BAED91B5BAFE2FFF73B5BAE078E0608F
:105F1000B5BA099400000000000000000000000075
:105F2000B5BAED91B5BAFE2FFF73B5BAE078E0616E
:105F3000B5BA099400000000000000000000000055
:105F4000B5BAED91B5BAFE2FFF73B5BAE078E0624D
:105F5000B5BA099400000000000000000000000035
:105F6000B5BAED91B5BAFE2FFF73B5BAE078E0632C
:105F7000B5BA099400000000000000000000000015
:105F8000B5BAED91B5BAFE2FFF73B5BAE078E0640B
:105F9000B5BA0994000000000000000000000000F5
:105FA000B5BAED91B5BAFE2FFF73B5BAE078E065EA
:105FB000B5BA0994000000000000000000000000D5
:105FC000B5BAED91B5BAFE2FFF73B5BAE078E066C9
:105FD000B5BA0994000000000000000000000000B5
:105FE000A5BAED91A5BAFE2FFF73A5BAE078E067D8
:105FF000B5BA099400000000000000000000000095
:10600000B5BAED91B5BAFE2FFF73B5BAE078E0608E
:10601000B5BA099400000000000000000000000074
:10602000B5BAED91A5BAFE2FFF73B5BAE078E0617D
:10603000B5BA099400000000000000000000000054
:10604000B5BAED91B5BAFE2FFF73A5BAE078E0625C
:10605000B5BA099400000000000000000000000034
:10606000B5BAED91B5BAFE2FFF73B5BAE078E0632B
:10607000B5BA099400000000000000000000000014
:10608000B5BAED91B5BAFE2FFF73B5BAE078E0640A
:10609000B5BA0994000000000000000000000000F4
:1060A000B5BAED91B5BAFE2FFF73B5BAE078E065E9
:1060B000B5BA0994000000000000000000000000D4
:1060C000B5BAED91B5BAFE2FFF73B5BAE078E066C8
:1060D000B5BA0994000000000000000000000000B4
:1060E000B5BAED91B5BAFE2FFF73B5BAE078E067A7
:1060F000B5BA099400000000000000000000000094
:10610000B5BAED91B5BAFE2FFF73B5BAE078E0608D
:10611000B5BA099400000000000000000000000073
:10612000B5BAED91B5BAFE2FFF73B5BAE078E0616C
:10613000B5BA099400000000000000000000000053
:10614000B5BAED91B5BAFE2FFF73B5BAE078E0624B
:10615000B5BA099400000000000000000000000033
:10616000B5BAED91A5BAFE2FFF73A5BAE078E0634A
:10617000B5BA099400000000000000000000000013
:10618000A5BAED91B5BAFE2FFF73A5BAE078E06429
:10619000B5BA0994000000000000000000000000F3
:1061A000A5BAED91B5BAFE2FFF73A5BAE078E06508
:1061B000B5BA0994000000000000000000000000D3
:1061C000B5BAED91A5BAFE2FFF73A5BAE078E066E7
:1061D000B5BA0994000000000000000000000000B3
:1061E000B5BAED91B5BAFE2FFF73B5BAE078E067A6
:1061F000B5BA099400000000000000000000000093
:10620000B5BAED91B5BAFE2FFF73B5BAE078E0608C
:10621000B5BA099400000000000000000000000072
:10622000A5BAED91B5BAFE2FFF73B5BAE078E0617B
:10623000B5BA099400000000000000000000000052
:10624000A5BAED91B5BAFE2FFF73B5BAE078E0625A
:10625000B5BA099400000000000000000000000032
:10626000A5BAED91A5BAFE2FFF73B5BAE078E06349
:10627000B5BA099400000000000000000000000012
:10628000A5BAED91B5BAFE2FFF73A5BAE078E06428
:10629000B5BA0994000000000000000000000000F2
:1062A000A5BAED91B5BAFE2FFF73A5BAE078E06507
:1062B000B5BA0994000000000000000000000000D2
:1062C000A5BAED91A5BAFE2FFF73B5BAE078E066E6
:1062D000B5BA0994000000000000000000000000B2
:1062E000B5BAED91B5BAFE2FFF73B5BAE078E067A5
:1062F000B5BA099400000000000000000000000092
:10630000B5BAED91B5BAFE2FFF73B5BAE078E0608B
:10631000B5BA099400000000000000000000000071
:10632000B5BAED91B5BAFE2FFF73B5BAE078E0616A
:10633000B5BA099400000000000000000000000051
:10634000B5BAED91B5BAFE2FFF73B5BAE078E06249
:10635000B5BA099400000000000000000000000031
:10636000B5BAED91A5BAFE2FFF73A5BAE078E06348
:10637000B5BA099400000000000000000000000011
:10638000A5BAED91B5BAFE2FFF73B5BAE078E06417
:10639000B5BA0994000000000000000000000000F1
:1063A000A5BAED91B5BAFE2FFF73B5BAE078E065F6
:1063B000B5BA0994000000000000000000000000D1
:1063C000B5BAED91A5BAFE2FFF73A5BAE078E066E5
:1063D000B5BA0994000000000000000000000000B1
:1063E000B5BAED91B5BAFE2FFF73B5BAE078E067A4
:1063F000B5BA099400000000000000000000000091
:10640000B5BAED91B5BAFE2FFF73B5BAE078E0608A
:10641000B5BA099400000000000000000000000070
:10642000B5BAED91B5BAFE2FFF73A5BAE078E06179
:10643000B5BA099400000000000000000000000050
:10644000B5BAED91B5BAFE2FFF73A5BAE078E06258
:10645000B5BA099400000000000000000000000030
:10646000B5BAED91A5BAFE2FFF73A5BAE078E06347
:10647000B5BA099400000000000000000000000010
:10648000A5BAED91B5BAFE2FFF73A5BAE078E06426
:10649000B5BA0994000000000000000000000000F0
:1064A000A5BAED91B5BAFE2FFF73A5BAE078E06505
:1064B000B5BA0994000000000000000000000000D0
:1064C000B5BAED91A5BAFE2FFF73A5BAE078E066E4
:1064D000B5BA0994000000000000000000000000B0
:1064E000B5BAED91B5BAFE2FFF73B5BAE078E067A3
:1064F000B5BA099400000000000000000000000090
:10650000B5BAED91B5BAFE2FFF73B5BAE078E06089
:10651000B5BA09940000000000000000000000006F
:10652000B5BAED91B5BAFE2FFF73B5BAE078E06168
:10653000B5BA09940000000000000000000000004F
:10654000B5BAED91B5BAFE2FFF73B5BAE078E06247
:10655000B5BA09940000000000000000000000002F
:10656000B5BAED91A5BAFE2FFF73B5BAE078E06336
:10657000B5BA09940000000000000000000000000F
:10658000A5BAED91B5BAFE2FFF73A5BAE078E06425
:10659000B5BA0994000000000000000000000000EF
:1065A000A5BAED91A5BAFE2FFF73B5BAE078E06504
:1065B000B5BA0994000000000000000000000000CF
:1065C000B5BAED91A5BAFE2FFF73A5BAE078E066E3
:1065D000B5BA0994000000000000000000000000AF
:1065E000B5BAED91B5BAFE2FFF73B5BAE078E067A2
:1065F000B5BA09940000000000000000000000008F
:10660000B5BAED91B5BAFE2FFF73B5BAE078E06088
:10661000B5BA09940000000000000000000000006E
:10662000B5BAED91B5BAFE2FFF73A5BAE078E06177
:10663000B5BA09940000000000000000000000004E
:10664000B5BAED91A5BAFE2FFF73B5BAE078E06256
:10665000B5BA09940000000000000000000000002E
:10666000A5BAED91A5BAFE2FFF73A5BAE078E06355
:10667000B5BA09940000000000000000000000000E
:10668000B5BAED91A5BAFE2FFF73B5BAE078E06414
:10669000B5BA0994000000000000000000000000EE
:1066A000B5BAED91A5BAFE2FFF73B5BAE078E065F3
:1066B000B5BA0994000000000000000000000000CE
:1066C000B5BAED91A5BAFE2FFF73B5BAE078E066D2
:1066D000B5BA0994000000000000000000000000AE
:1066E000B5BAED91B5BAFE2FFF73B5BAE078E067A1
:1066F000B5BA09940000000000000000000000008E
:10670000B5BAED91B5BAFE2FFF73B5BAE078E06087
:10671000B5BA09940000000000000000000000006D
:10672000B5BAED91B5BAFE2FFF73B5BAE078E06166
:10673000B5BA09940000000000000000000000004D
:10674000B5BAED91B5BAFE2FFF73B5BAE078E06245
:10675000B5BA09940000000000000000000000002D
:10676000B5BAED91A5BAFE2FFF73A5BAE078E06344
:10677000B5BA09940000000000000000000000000D
:10678000A5BAED91B5BAFE2FFF73A5BAE078E06423
:10679000B5BA0994000000000000000000000000ED
:1067A000B5BAED91A5BAFE2FFF73A5BAE078E06502
:1067B000B5BA0994000000000000000000000000CD
:1067C000B5BAED91B5BAFE2FFF73A5BAE078E066D1
:1067D000B5BA0994000000000000000000000000AD
:1067E000A5BAED91A5BAFE2FFF73B5BAE078E067C0
:1067F000B5BA09940000000000000000000000008D
:10680000B5BAED91B5BAFE2FFF73B5BAE078E06086
:10681000B5BA09940000000000000000000000006C
:10682000A5BAED91B5BAFE2FFF73B5BAE078E06175
:10683000B5BA09940000000000000000000000004C
:10684000A5BAED91B5BAFE2FFF73B5BAE078E06254
:10685000B5BA09940000000000000000000000002C
:10686000A5BAED91A5BAFE2FFF73B5BAE078E06343
:10687000B5BA09940000000000000000000000000C
:10688000A5BAED91B5BAFE2FFF73A5BAE078E06422
:10689000B5BA0994000000000000000000000000EC
:1068A000A5BAED91B5BAFE2FFF73A5BAE078E06501
:1068B000B5BA0994000000000000000000000000CC
:1068C000A5BAED91B5BAFE2FFF73A5BAE078E066E0
:1068D000B5BA0994000000000000000000000000AC
:1068E000B5BAED91B5BAFE2FFF73B5BAE078E0679F
:1068F000B5BA09940000000000000000000000008C
:10690000B5BAED91B5BAFE2FFF73B5BAE078E06085
:10691000B5BA09940000000000000000000000006B
:10692000B5BAED91A5BAFE2FFF73B5BAE078E06174
:10693000B5BA09940000000000000000000000004B
:10694000B5BAED91B5BAFE2FFF73B5BAE078E06243
:10695000B5BA09940000000000000000000000002B
:10696000A5BAED91A5BAFE2FFF73B5BAE078E06342
:10697000B5BA09940000000000000000000000000B
:10698000B5BAED91A5BAFE2FFF73B5BAE078E06411
:10699000B5BA0994000000000000000000000000EB
:1069A000B5BAED91A5BAFE2FFF73B5BAE078E065F0
:1069B000B5BA0994000000000000000000000000CB
:1069C000A5BAED91A5BAFE2FFF73A5BAE078E066EF
:1069D000B5BA0994000000000000000000000000AB
:1069E000B5BAED91B5BAFE2FFF73B5BAE078E0679E
:1069F000B5BA09940000000000000000000000008B
:106A0000B5BAED91B5BAFE2FFF73B5BAE078E06084
:106A1000B5BA09940000000000000000000000006A
:106A2000B5BAED91A5BAFE2FFF73B5BAE078E06173
:106A3000B5BA09940000000000000000000000004A
:106A4000B5BAED91B5BAFE2FFF73B5BAE078E06242
:106A5000B5BA09940000000000000000000000002A
:106A6000A5BAED91A5BAFE2FFF73B5BAE078E06341
:106A7000B5BA09940000000000000000000000000A
:106A8000B5BAED91A5BAFE2FFF73B5BAE078E06410
:106A9000B5BA0994000000000000000000000000EA
:106AA000B5BAED91A5BAFE2FFF73B5BAE078E065EF
:106AB000B5BA0994000000000000000000000000CA
:106AC000B5BAED91A5BAFE2FFF73B5BAE078E066CE
:106AD000B5BA0994000000000000000000000000AA
:106AE000A5BAED91B5BAFE2FFF73B5BAE078E067AD
:106AF000B5BA09940000000000000000000000008A
:106B0000B5BAED91B5BAFE2FFF73B5BAE078E06083
:106B1000B5BA099400000000000000000000000069
:106B2000A5BAED91B5BAFE2FFF73B5BAE078E06172
:106B3000B5BA099400000000000000000000000049
:106B4000A5BAED91B5BAFE2FFF73B5BAE078E06251
:106B5000B5BA099400000000000000000000000029
:106B6000A5BAED91B5BAFE2FFF73A5BAE078E06340
:106B7000B5BA099400000000000000000000000009
:106B8000A5BAED91A5BAFE2FFF73B5BAE078E0641F
:106B9000B5BA0994000000000000000000000000E9
:106BA000A5BAED91A5BAFE2FFF73B5BAE078E065FE
:106BB000B5BA0994000000000000000000000000C9
:106BC000A5BAED91B5BAFE2FFF73A5BAE078E066DD
:106BD000B5BA0994000000000000000000000000A9
:106BE000B5BAED91B5BAFE2FFF73B5BAE078E0679C
:106BF000B5BA099400000000000000000000000089
:106C0000B5BAED91B5BAFE2FFF73B5BAE078E06082
:106C1000B5BA099400000000000000000000000068
:106C2000A5BAED91A5BAFE2FFF73B5BAE078E06181
:106C3000B5BA099400000000000000000000000048
:106C4000B5BAED91A5BAFE2FFF73B5BAE078E06250
:106C5000B5BA099400000000000000000000000028
:106C6000B5BAED91A5BAFE2FFF73B5BAE078E0632F
:106C7000B5BA099400000000000000000000000008
:106C8000B5BAED91A5BAFE2FFF73B5BAE078E0640E
:106C9000B5BA0994000000000000000000000000E8
:106CA000B5BAED91A5BAFE2FFF73B5BAE078E065ED
:106CB000B5BA0994000000000000000000000000C8
:106CC000A5BAED91A5BAFE2FFF73A5BAE078E066EC
:106CD000B5BA0994000000000000000000000000A8
:106CE000B5BAED91B5BAFE2FFF73B5BAE078E0679B
:106CF000B5BA099400000000000000000000000088
:106D0000B5BAED91B5BAFE2FFF73B5BAE078E06081
:106D1000B5BA099400000000000000000000000067
:106D2000B5BAED91B5BAFE2FFF73B5BAE078E06160
:106D3000B5BA099400000000000000000000000047
:106D4000B5BAED91B5BAFE2FFF73B5BAE078E0623F
:106D5000B5BA099400000000000000000000000027
:106D6000A5BAED91A5BAFE2FFF73B5BAE078E0633E
:106D7000B5BA099400000000000000000000000007
:106D8000A5BAED91A5BAFE2FFF73A5BAE078E0642D
:106D9000B5BA0994000000000000000000000000E7
:106DA000A5BAED91A5BAFE2FFF73A5BAE078E0650C
:106DB000B5BA0994000000000000000000000000C7
:106DC000A5BAED91A5BAFE2FFF73A5BAE078E066EB
:106DD000B5BA0994000000000000000000000000A7
:106DE000B5BAED91B5BAFE2FFF73B5BAE078E0679A
:106DF000B5BA099400000000000000000000000087
:106E0000B5BAED91B5BAFE2FFF73B5BAE078E06080
:106E1000B5BA099400000000000000000000000066
:106E2000B5BAED91B5BAFE2FFF73B5BAE078E0615F
:106E3000B5BA099400000000000000000000000046
:106E4000B5BAED91B5BAFE2FFF73B5BAE078E0623E
:106E5000B5BA099400000000000000000000000026
:106E6000A5BAED91A5BAFE2FFF73B5BAE078E0633D
:106E7000B5BA099400000000000000000000000006
:106E8000A5BAED91B5BAFE2FFF73A5BAE078E0641C
:106E9000B5BA0994000000000000000000000000E6
:106EA000A5BAED91B5BAFE2FFF73A5BAE078E065FB
:106EB000B5BA0994000000000000000000000000C6
:106EC000A5BAED91B5BAFE2FFF73A5BAE078E066DA
:106ED000B5BA0994000000000000000000000000A6
:106EE000B5BAED91B5BAFE2FFF73B5BAE078E06799
:106EF000B5BA099400000000000000000000000086
:106F0000B5BAED91B5BAFE2FFF73B5BAE078E0607F
:106F1000B5BA099400000000000000000000000065
:106F2000B5BAED91B5BAFE2FFF73B5BAE078E0615E
:106F3000B5BA099400000000000000000000000045
:106F4000B5BAED91B5BAFE2FFF73B5BAE078E0623D
:106F5000B5BA099400000000000000000000000025
:106F6000B5BAED91A5BAFE2FFF73B5BAE078E0632C
:106F7000B5BA099400000000000000000000000005
:106F8000A5BAED91B5BAFE2FFF73A5BAE078E0641B
:106F9000B5BA0994000000000000000000000000E5
:106FA000A5BAED91B5BAFE2FFF73A5BAE078E065FA
:106FB000B5BA0994000000000000000000000000C5
:106FC000B5BAED91A5BAFE2FFF73B5BAE078E066C9
:106FD000B5BA0994000000000000000000000000A5
:106FE000B5BAED91B5BAFE2FFF73B5BAE078E06798
:106FF000B5BA099400000000000000000000000085
:10700000B5BAED91B5BAFE2FFF73B5BAE078E0607E
:10701000B5BA099400000000000000000000000064
:10702000B5BAED91B5BAFE2FFF73B5BAE078E0615D
:10703000B5BA099400000000000000000000000044
:10704000B5BAED91B5BAFE2FFF73B5BAE078E0623C
:10705000B5BA099400000000000000000000000024
:10706000A5BAED91A5BAFE2FFF73B5BAE078E0633B
:10707000B5BA099400000000000000000000000004
:10708000A5BAED91B5BAFE2FFF73A5BAE078E0641A
:10709000B5BA0994000000000000000000000000E4
:1070A000A5BAED91A5BAFE2FFF73B5BAE078E065F9
:1070B000B5BA0994000000000000000000000000C4
:1070C000A5BAED91B5BAFE2FFF73B5BAE078E066C8
:1070D000B5BA0994000000000000000000000000A4
:1070E000A5BAED91B5BAFE2FFF73B5BAE078E067A7
:1070F000B5BA099400000000000000000000000084
:10710000B5BAED91B5BAFE2FFF73B5BAE078E0607D
:10711000B5BA099400000000000000000000000063
:10712000B5BAED91B5BAFE2FFF73B5BAE078E0615C
:10713000B5BA099400000000000000000000000043
:10714000B5BAED91B5BAFE2FFF73B5BAE078E0623B
:10715000B5BA099400000000000000000000000023
:10716000B5BAED91A5BAFE2FFF73A5BAE078E0633A
:10717000B5BA099400000000000000000000000003
:10718000A5BAED91B5BAFE2FFF73A5BAE078E06419
:10719000B5BA0994000000000000000000000000E3
:1071A000B5BAED91A5BAFE2FFF73A5BAE078E065F8
:1071B000B5BA0994000000000000000000000000C3
:1071C000B5BAED91B5BAFE2FFF73A5BAE078E066C7
:1071D000B5BA0994000000000000000000000000A3
:1071E000B5BAED91B5BAFE2FFF73A5BAE078E067A6
:1071F000B5BA099400000000000000000000000083
:10720000B5BAED91B5BAFE2FFF73B5BAE078E0607C
:10721000B5BA099400000000000000000000000062
:10722000B5BAED91B5BAFE2FFF73B5BAE078E0615B
:10723000B5BA099400000000000000000000000042
:10724000B5BAED91B5BAFE2FFF73B5BAE078E0623A
:10725000B5BA099400000000000000000000000022
:10726000A5BAED91A5BAFE2FFF73B5BAE078E06339
:10727000B5BA099400000000000000000000000002
:10728000A5BAED91B5BAFE2FFF73A5BAE078E06418
:10729000B5BA0994000000000000000000000000E2
:1072A000A5BAED91B5BAFE2FFF73B5BAE078E065E7
:1072B000B5BA0994000000000000000000000000C2
:1072C000A5BAED91B5BAFE2FFF73B5BAE078E066C6
:1072D000B5BA0994000000000000000000000000A2
:1072E000B5BAED91B5BAFE2FFF73B5BAE078E06795
:1072F000B5BA099400000000000000000000000082
:10730000B5BAED91B5BAFE2FFF73B5BAE078E0607B
:10731000B5BA099400000000000000000000000061
:10732000B5BAED91B5BAFE2FFF73B5BAE078E0615A
:10733000B5BA099400000000000000000000000041
:10734000B5BAED91B5BAFE2FFF73B5BAE078E06239
:10735000B5BA099400000000000000000000000021
:10736000B5BAED91A5BAFE2FFF73A5BAE078E06338
:10737000B5BA099400000000000000000000000001
:10738000A5BAED91B5BAFE2FFF73B5BAE078E06407
:10739000B5BA0994000000000000000000000000E1
:1073A000B5BAED91A5BAFE2FFF73A5BAE078E065F6
:1073B000B5BA0994000000000000000000000000C1
:1073C000A5BAED91A5BAFE2FFF73B5BAE078E066D5
:1073D000B5BA0994000000000000000000000000A1
:1073E000B5BAED91B5BAFE2FFF73B5BAE078E06794
:1073F000B5BA099400000000000000000000000081
:10740000B5BAED91B5BAFE2FFF73B5BAE078E0607A
:10741000B5BA099400000000000000000000000060
:10742000B5BAED91A5BAFE2FFF73B5BAE078E06169
:10743000B5BA099400000000000000000000000040
:10744000B5BAED91A5BAFE2FFF73B5BAE078E06248
:10745000B5BA099400000000000000000000000020
:10746000A5BAED91A5BAFE2FFF73A5BAE078E06347
:10747000B5BA099400000000000000000000000000
:10748000B5BAED91A5BAFE2FFF73B5BAE078E06406
:10749000B5BA0994000000000000000000000000E0
:1074A000B5BAED91A5BAFE2FFF73B5BAE078E065E5
:1074B000B5BA0994000000000000000000000000C0
:1074C000B5BAED91B5BAFE2FFF73A5BAE078E066C4
:1074D000B5BA0994000000000000000000000000A0
:1074E000B5BAED91B5BAFE2FFF73B5BAE078E06793
:1074F000B5BA099400000000000000000000000080
:10750000B5BAED91B5BAFE2FFF73B5BAE078E06079
:10751000B5BA09940000000000000000000000005F
:10752000B5BAED91B5BAFE2FFF73B5BAE078E06158
:10753000B5BA09940000000000000000000000003F
:10754000B5BAED91B5BAFE2FFF73B5BAE078E06237
:10755000B5BA09940000000000000000000000001F
:10756000A5BAED91B5BAFE2FFF73A5BAE078E06336
:10757000B5BA0994000000000000000000000000FF
:10758000A5BAED91B5BAFE2FFF73A5BAE078E06415
:10759000B5BA0994000000000000000000000000DF
:1075A000A5BAED91B5BAFE2FFF73A5BAE078E065F4
:1075B000B5BA0994000000000000000000000000BF
:1075C000B5BAED91A5BAFE2FFF73A5BAE078E066D3
:1075D000B5BA09940000000000000000000000009F
:1075E000B5BAED91B5BAFE2FFF73B5BAE078E06792
:1075F000B5BA09940000000000000000000000007F
:10760000B5BAED91B5BAFE2FFF73B5BAE078E06078
:10761000B5BA09940000000000000000000000005E
:10762000B5BAED91B5BAFE2FFF73B5BAE078E06157
:10763000B5BA09940000000000000000000000003E
:10764000B5BAED91B5BAFE2FFF73B5BAE078E06236
:10765000B5BA09940000000000000000000000001E
:10766000A5BAED91B5BAFE2FFF73A5BAE078E06335
:10767000B5BA0994000000000000000000000000FE
:10768000A5BAED91B5BAFE2FFF73A5BAE078E06414
:10769000B5BA0994000000000000000000000000DE
:1076A000B5BAED91A5BAFE2FFF73B5BAE078E065E3
:1076B000B5BA0994000000000000000000000000BE
:1076C000B5BAED91A5BAFE2FFF73B5BAE078E066C2
:1076D000B5BA09940000000000000000000000009E
:1076E000B5BAED91B5BAFE2FFF73B5BAE078E06791
:1076F000B5BA09940000000000000000000000007E
:10770000B5BAED91B5BAFE2FFF73B5BAE078E06077
:10771000B5BA09940000000000000000000000005D
:10772000B5BAED91B5BAFE2FFF73B5BAE078E06156
:10773000B5BA09940000000000000000000000003D
:10774000B5BAED91B5BAFE2FFF73B5BAE078E06235
:10775000B5BA09940000000000000000000000001D
:10776000A5BAED91B5BAFE2FFF73A5BAE078E06334
:10777000B5BA0994000000000000000000000000FD
:10778000A5BAED91B5BAFE2FFF73A5BAE078E06413
:10779000B5BA0994000000000000000000000000DD
:1077A000A5BAED91A5BAFE2FFF73A5BAE078E06502
:1077B000B5BA0994000000000000000000000000BD
:1077C000A5BAED91A5BAFE2FFF73A5BAE078E066E1
:1077D000B5BA09940000000000000000000000009D
:1077E000B5BAED91B5BAFE2FFF73B5BAE078E06790
:1077F000B5BA09940000000000000000000000007D
:10780000B5BAED91B5BAFE2FFF73B5BAE078E06076
:10781000B5BA09940000000000000000000000005C
:10782000B5BAED91B5BAFE2FFF73B5BAE078E06155
:10783000B5BA09940000000000000000000000003C
:10784000B5BAED91B5BAFE2FFF73B5BAE078E06234
:10785000B5BA09940000000000000000000000001C
:10786000A5BAED91B5BAFE2FFF73A5BAE078E06333
:10787000B5BA0994000000000000000000000000FC
:10788000B5BAED91A5BAFE2FFF73B5BAE078E06402
:10789000B5BA0994000000000000000000000000DC
:1078A000B5BAED91A5BAFE2FFF73B5BAE078E065E1
:1078B000B5BA0994000000000000000000000000BC
:1078C000A5BAED91B5BAFE2FFF73A5BAE078E066D0
:1078D000B5BA09940000000000000000000000009C
:1078E000B5BAED91B5BAFE2FFF73B5BAE078E0678F
:1078F000B5BA09940000000000000000000000007C
:10790000B5BAED91B5BAFE2FFF73B5BAE078E06075
:10791000B5BA09940000000000000000000000005B
:10792000B5BAED91B5BAFE2FFF73B5BAE078E06154
:10793000B5BA09940000000000000000000000003B
:10794000B5BAED91B5BAFE2FFF73B5BAE078E06233
:10795000B5BA09940000000000000000000000001B
:10796000A5BAED91B5BAFE2FFF73A5BAE078E06332
:10797000B5BA0994000000000000000000000000FB
:10798000A5BAED91B5BAFE2FFF73A5BAE078E06411
:10799000B5BA0994000000000000000000000000DB
:1079A000B5BAED91A5BAFE2FFF73A5BAE078E065F0
:1079B000B5BA0994000000000000000000000000BB
:1079C000B5BAED91B5BAFE2FFF73A5BAE078E066BF
:1079D000B5BA09940000000000000000000000009B
:1079E000A5BAED91A5BAFE2FFF73B5BAE078E067AE
:1079F000B5BA09940000000000000000000000007B
:107A0000B5BAED91B5BAFE2FFF73B5BAE078E06074
:107A1000B5BA09940000000000000000000000005A
:107A2000B5BAED91B5BAFE2FFF73B5BAE078E06153
:107A3000B5BA09940000000000000000000000003A
:107A4000B5BAED91B5BAFE2FFF73B5BAE078E06232
:107A5000B5BA09940000000000000000000000001A
:107A6000A5BAED91A5BAFE2FFF73A5BAE078E06341
:107A7000B5BA0994000000000000000000000000FA
:107A8000B5BAED91A5BAFE2FFF73B5BAE078E06400
:107A9000B5BA0994000000000000000000000000DA
:107AA000A5BAED91B5BAFE2FFF73B5BAE078E065DF
:107AB000B5BA0994000000000000000000000000BA
:107AC000A5BAED91A5BAFE2FFF73A5BAE078E066DE
:107AD000B5BA09940000000000000000000000009A
:107AE000B5BAED91B5BAFE2FFF73B5BAE078E0678D
:107AF000B5BA09940000000000000000000000007A
:107B0000B5BAED91B5BAFE2FFF73B5BAE078E06073
:107B1000B5BA099400000000000000000000000059
:107B2000B5BAED91A5BAFE2FFF73A5BAE078E06172
:107B3000B5BA099400000000000000000000000039
:107B4000B5BAED91A5BAFE2FFF73B5BAE078E06241
:107B5000B5BA099400000000000000000000000019
:107B6000A5BAED91A5BAFE2FFF73B5BAE078E06330
:107B7000B5BA0994000000000000000000000000F9
:107B8000B5BAED91A5BAFE2FFF73B5BAE078E064FF
:107B9000B5BA0994000000000000000000000000D9
:107BA000B5BAED91A5BAFE2FFF73B5BAE078E065DE
:107BB000B5BA0994000000000000000000000000B9
:107BC000B5BAED91A5BAFE2FFF73A5BAE078E066CD
:107BD000B5BA099400000000000000000000000099
:107BE000B5BAED91B5BAFE2FFF73B5BAE078E0678C
:107BF000B5BA099400000000000000000000000079
:107C0000B5BAED91B5BAFE2FFF73B5BAE078E06072
:107C1000B5BA099400000000000000000000000058
:107C2000B5BAED91A5BAFE2FFF73B5BAE078E06161
:107C3000B5BA099400000000000000000000000038
:107C4000B5BAED91A5BAFE2FFF73B5BAE078E06240
:107C5000B5BA099400000000000000000000000018
:107C6000B5BAED91A5BAFE2FFF73B5BAE078E0631F
:107C7000B5BA0994000000000000000000000000F8
:107C8000B5BAED91A5BAFE2FFF73B5BAE078E064FE
:107C9000B5BA0994000000000000000000000000D8
:107CA000B5BAED91A5BAFE2FFF73B5BAE078E065DD
:107CB000B5BA0994000000000000000000000000B8
:107CC000B5BAED91A5BAFE2FFF73B5BAE078E066BC
:107CD000B5BA099400000000000000000000000098
:107CE000B5BAED91B5BAFE2FFF73B5BAE078E0678B
:107CF000B5BA099400000000000000000000000078
:107D0000B5BAED91B5BAFE2FFF73B5BAE078E06071
:107D1000B5BA099400000000000000000000000057
:107D2000A5BAED91A5BAFE2FFF73B5BAE078E06170
:107D3000B5BA099400000000000000000000000037
:107D4000B5BAED91A5BAFE2FFF73B5BAE078E0623F
:107D5000B5BA099400000000000000000000000017
:107D6000B5BAED91A5BAFE2FFF73A5BAE078E0632E
:107D7000B5BA0994000000000000000000000000F7
:107D8000B5BAED91A5BAFE2FFF73B5BAE078E064FD
:107D9000B5BA0994000000000000000000000000D7
:107DA000B5BAED91A5BAFE2FFF73B5BAE078E065DC
:107DB000B5BA0994000000000000000000000000B7
:107DC000A5BAED91A5BAFE2FFF73B5BAE078E066CB
:107DD000B5BA099400000000000000000000000097
:107DE000B5BAED91B5BAFE2FFF73B5BAE078E0678A
:107DF000B5BA099400000000000000000000000077
:107E0000B5BAED91B5BAFE2FFF73B5BAE078E06070
:107E1000B5BA099400000000000000000000000056
:107E2000B5BAED91A5BAFE2FFF73A5BAE078E0616F
:107E3000B5BA099400000000000000000000000036
:107E4000A5BAED91A5BAFE2FFF73B5BAE078E0624E
:107E5000B5BA099400000000000000000000000016
:107E6000B5BAED91B5BAFE2FFF73B5BAE078E0630D
:107E7000B5BA0994000000000000000000000000F6
:107E8000B5BAED91B5BAFE2FFF73B5BAE078E064EC
:107E9000B5BA0994000000000000000000000000D6
:107EA000B5BAED91B5BAFE2FFF73B5BAE078E065CB
:107EB000B5BA0994000000000000000000000000B6
:107EC000B5BAED91B5BAFE2FFF73B5BAE078E066AA
:107ED000B5BA099400000000000000000000000096
:107EE000B5BAED91B5BAFE2FFF73B5BAE078E06789
:107EF000B5BA099400000000000000000000000076
:107F0000F5BA0C941201000000000000000000000F
:107F10000000000000000000000000000000000061
:107F2000F5BA0C94120100000000000000000000EF
:107F30000000000000000000000000000000000041
:107F4000F5BA0C94120100000000000000000000CF
:107F50000000000000000000000000000000000021
:107F6000F5BA0C94120100000000000000000000AF
:107F70000000000000000000000000000000000001
:107F8000F5BA0C941201000000000000000000008F
:107F900000000000000000000000000000000000E1
:107FA000F5BA0C941201000000000000000000006F
:107FB00000000000000000000000000000000000C1
:107FC000F5BA0C941201000000000000000000004F
:107FD00000000000000000000000000000000000A1
:107FE000F5BA0C941201000000000000000000002F
:107FF0000000000000000000000000000000000081
:00000001FF
